:10587600126561126F2B306D2353B1F8C26D12722F
:10588600961273ED12712C126D7D1265131267B7A5
:10589600126F5B1258EE124D5F127282306C22C28A
:1058A6006C121C7A125DF91271F812716912718606
:1058B600125D30400312515712726D124531125368
:1058C600C2126F881271A31263881246C8124E0C58
:1058D600126C0B900206E524F0A3E525F0A3E52261
:0858E600F0A3E523F0808C2201
:106B48009005367401F07E027F3C7B40E4FD126FB5
:106B5800DF7E027F0A7B14E4126FDF900224740A3E
:106B6800F0A374ABF0A3740AF0A374ABF0C22CC208
:106B78002D90053F7402F0D22ED27B90027C745087
:026B8800F022F9
:105157007FFE7E01127009501F7B007A02E4FDFC7E
:10516700FFFE125F187FFE7E03127009402CE4FDDC
:10517700FF7E0212532B80227FFE7E03127009509E
:10518700167B007A02E4FDFCFF7E02125F18E4FD45
:10519700FFFE12532B8003D26E22900000E0F52011
:1051A700A3E0F521900238E520F0A3E521F0900077
:1051B7001A12259A90022C122600900022E0FFA3D3
:1051C700E0900236CFF0A3EFF0E52154072403F572
:1051D7001364056005E513B40A04E4F51422E51326
:1051E70064046005E513B4090475140122751402FB
:0151F7002295
:10714B00C2AFD2ACC086758640C28FD086D2AD435B
:0E715B00BA6043E840E4F5D843A908D2AF2259
:106FB40075803875E10F75E90875908075E27F7505
:106FC400EA8075A0E075E33F75EBC075B01975E410
:0B6FD400E675EC194380C043E9802201
:10656100E4FF126295126FB4125157126B487D0508
:106571007C007F44123EEC1271DC1272417D647F1B
:10658100A07E0F1257781255F01255694002D25A67
:10659100126D063007121257F94002D2397E047F7C
:0C65A100971254504002D27812714B2225
:10102E00EFB4200E206303306619E4FF126295D2EE
:10103E006522EFB4400D206303306607E4FF1262B1
:04104E0095D26522B0
:1070C900D26B9003FFE004F0C3940A4004E4F0D2C9
:1070D9006D9003FEE004F0C394C84004E4F0D26C60
:0470E9001250B5226A
:106C4B00D3EF9450EE940040037F0522D3EF943C96
:106C5B00EE940040037F0422D3EF9428EE9400407F
:106C6B00037F0322D3EF9414EE940040037F0222A0
:0F6C7B00D3EF9400EE940040037F01227F0022AC
:1072AA0030710F90053EE004F0C394644004E4F0AA
:0372BA00C271227C
:104D5F00302A1490053CE004F0C3940A400BE4F0B1
:104D6F00A2B5B392B58002C2B530721490053DE082
:104D7F0004F0C39405400BE4F0A2A0B392A080020C
:104D8F00C2A0307167900234E0FEA3E0FF126C4BBB
:104D9F00EF700D207202C2A0C2A1C2A2C2A3C2A410
:104DAF00EFB40107207252D2A0804EEFB402092057
:104DBF007202D2A0D2A18041EFB4030B207202D2B3
:104DCF00A0D2A1D2A28032EFB4040D207202D2A0E1
:104DDF00D2A1D2A2D2A38021EF6405701C2072024F
:104DEF00D2A0D2A1D2A2D2A3D2A4800D207202C28D
:0C4DFF00A0C2A1C2A2C2A3C2A41272AA48
:014E0B002284
:105CCA00C22CC22DC22E302B5690053FE07018040C
:105CDA00F0D22D900089E0FEA3E0FF90008CE0FD59
:105CEA0012577843B7012290053FE0B401167402B7
:105CFA00F0D22E900089E0FEA3E0FF7D641257786F
:105D0A0043B70122E490053FF0D22C900089E0FECF
:105D1A00A3E0FF90008BE0FD12577843B70122C23F
:065D2A002CC22DC22E2246
:106F2B00307A2CC27AE50824FE600F24F160161427
:106F3B00601024117019125CCA22D271E490053EC4
:106F4B00F022D26322B272307203C28322D2832226
:106BCB0030653CC265306624E4FF126295D2AFC2D9
:106BDB0066E49005E8F07F01126890D2ACD2ADD29A
:106BEB00CE7F7012722A12737B127309E49005E840
:106BFB00F0A3F09003F6F09003F7F09003F8F02277
:10710D0053B1F8C2AF207202C2A0C2A1C2A2C2A3E3
:0F711D00C2A4D283E4FF12725812705780E2228C
:106B0500207202C2A0C2A1C2A2C2A3C2A4D283C2E1
:106B15007212731C12738E7F701273B3C2CE53B789
:106B25007E302904D2A58002C2A57F01126890C2D9
:106B3500AFC2ACC2ADE4F5D87F80126295D2AF1278
:036B450073E122D7
:1053C20030640E204306204403304505C264D26394
:1053D2002230161490002AE0FF9005E9E004F0C3A1
:1053E2009F406AEFF0D2632220715B202A50202B6B
:1053F2004D30191490002AE0FF9005E9E004F0C353
:105402009F404AEFF0D26322E49005E9F0A21272C3
:10541200107218721A721172137219721B721C7244
:10542200157272401390002AE0FF9005E8E004F044
:105432009F401AEFF0D26622E49005E8F022E49051
:0E54420005E8F0A3F022E49005E8F0A3F022C4
:106C0B00206626206323C2AFA279727A726F7265F7
:106C1B00724C726D726C400D9005EAE06412600567
:106C2B00D2AF1273D5D2AF801330630AD26F124634
:106C3B00C812710D8006306603126B05126BCB22E6
:10680000000000300062007400000089008E0099D2
:1068100000A200AA00BB00BF00FE000000000000B4
:10682000000000000020005000820094000000A939
:1068300000AE00B900C200CA00DB00DF011E00008C
:08684000000000000000000050
:1073A100900402E07006C29C75995A22C29C75999C
:0273B100FF22B9
:085964009002B7EEF0A3EFF092
:10596C007B017A047900900402E02403FD1271C0DB
:10597C00900402E02403F582E43404F583E06F70B4
:10598C0041FF900402E0FEEFC39E502953B1F8741E
:10599C00032FF582E43404F583E0FE9002B7E0FCBB
:1059AC00A3E0F5828C83EEF09002B7E475F001125F
:1059BC0023C40F80CDD270E49005F3F0C29C75998E
:0759CC005A22C29C7599FFED
:0159D30022B1
:105D9600900402E0D3948C4002E4F0E4FD90040207
:105DA600E0FCEDC39C501D53B1F88F828E83E0FB5F
:105DB60074032DF582E43404F583EBF00FBF000184
:105DC6000E0D80D97B017A047900EC2403FD127153
:105DD600C0900402E02403F582E43404F583EFF076
:105DE600C29C9003F9E02400F582E43404F583E0D4
:025DF600F5991D
:015DF8002288
:1069AE007B017A047900900402E02403FD1271C089
:1069BE00900402E02403F582E43404F583E0B50785
:1069CE001E900404E0FFB441089005EA7412F080B2
:1069DE0006EFB40502D264C243C29C75995A22C214
:0569EE009C7599FF22D9
:106DB8007B017A047900900402E02403FD1271C07B
:106DC800900402E02403F582E43404F583E0B50777
:106DD80010900403E09003F1F0C243C29C75995AE5
:076DE80022C29C7599FF22F5
:1039CF00900401E0FF1226623A23013A23023A23C0
:1039DF00033A23043A23053A23063A23073A2308E6
:1039EF003A23093A230A3A340B3A440C3A4C0D3A2B
:1039FF00540E3A5C0F3A3C103A64113A6C123A7416
:103A0F00133A7C143A84153A8C163A94173A9C1848
:103A1F0000003AA4EF25E02408F582E43402AF82D7
:103A2F00FE125D96227E027F1E125D96227E027F1F
:103A3F0020125D96227E027F24125D96227E027FE7
:103A4F0026125D96227E027F28125D96227E027FCD
:103A5F002A125D96227E027F2C125D96227E027FB5
:103A6F0030125D96227E027F34125D96227E027F97
:103A7F0036125D96227E027F06125D96227E027FAF
:103A8F0008125D96227E027F38125D96227E027F9B
:103A9F003A125D9622900402E0C394804009D23A14
:103AAF009003E17401F022900401E0B478109003C8
:103ABF00F1E0B40C09D23A9003EE7401F0229004B5
:103ACF0001E0B478229003F1E025E02400F582E4D0
:103ADF003468F583E493FE740193FF9002B5EEF022
:103AEF00A3EFF0125D9622900401E0B479219003C8
:103AFF00F1E025E02424F582E43468F583E493FEB5
:0F3B0F00740193FF9002B5EEF0A3EFF0125D96F4
:013B1E002284
:106243007B017A047900900402E02403FD1271C0FB
:10625300900402E02403F582E43404F583E06F70D4
:106263002B900403E0FEA3E0FDEEEDFF9005DFEECF
:10627300F0A3EFF04E7006C29C7599FF22D279907D
:1062830005DAE04401F0C29C75995A22C29C7599C3
:02629300FF22E8
:104789007B017A047900900402E02403FD1271C0D0
:10479900900402E02403F582E43404F583E06F60B9
:1047A90003024840900404E0FFE4FCFDFE78101287
:1047B900257BC004C005C006C007900403E0FFE4E0
:1047C900FCFDFE781812257BD003D002D001D00061
:1047D900122512C004C005C006C007900405E0FFF9
:1047E900E4FCFDFE780812257BD003D002D001D06D
:1047F90000122512A804A905AA06AB07A3E0FFE445
:10480900FCFDFE1225129005D61226009002A1E0A9
:104819007002A3E0600C9005D612259AEC4D4E4F1C
:104829007006C29C7599FF22D2799005DAE044108E
:0D483900F0C29C75995A22C29C7599FF220D
:106DEF007B017A047900900402E02403FD1271C044
:106DFF00900402E02403F582E43404F583E0B50740
:106E0F000FD2799005DAE04420F0C29C75995A228E
:066E1F00C29C7599FF22E0
:106725007B017A047900900402E02403FD1271C014
:10673500900402E02403F582E43404F583E06F70ED
:1067450022D279900403E0FEA3E0FDEEEDFF900573
:10675500DBEEF0A3EFF09005DAE04404F0C29C759F
:09676500995A22C29C7599FF2289
:10676E007B017A047900900402E02403FD1271C0CB
:10677E00900402E02403F582E43404F583E06F70A4
:10678E0022D279900403E0FEA3E0FDEEEDFF90052A
:10679E00DDEEF0A3EFF09005DAE04408F0C29C7550
:0967AE00995A22C29C7599FF2240
:1061EF007B017A047900900402E02403FD1271C050
:1061FF00900402E02403F582E43404F583E06F7029
:10620F002DFF74032FF582E43404F583E0FE74E16F
:10621F002FF582E43405F583EEF00FEFB407E3D2E8
:10622F00799005DAE04480F0C29C75995A22C29C9D
:03623F007599FF4F
:016242002239
:10500E00900401E0122662503A18503E77505A78BA
:10501E00507C795046A0504EA15052A25042A350FF
:10502E004AA45056AF509EB0000050B41269AE2242
:10503E00126DB8221247892212624322126DEF229C
:10504E001267252212676E221261EF229003F1E0A1
:10505E0025E02400F582E43468F583E493FE7401C0
:10506E0093FF9002B5EEF0A3EFF012596422900375
:10507E00F1E025E02424F582E43468F583E493FE20
:10508E00740193FF9002B5EEF0A3EFF01259642273
:10509E00900403E0B4550AD23AD238C29C75995A9C
:0650AE0022C29C7599FF6F
:0150B40022D9
:10386800E49002B5F0A3F09003F9E0FFB4021A90D7
:103878000401E064A56006E49003F9F022E49003F3
:10388800FCF0A3F09003F2F022900402E0FD7C002B
:103898002409FBEC33FA7E00C3EF9BEA6480F874DA
:1038A8008098505FED2407FDEC33FCD3EF9DEC646A
:1038B80080F874809850189003F9E024FFF582E4AA
:1038C8003403F583E0FF9003FCEE8FF01223C490DD
:1038D80003F9E0FFB40511900404E06407700302E3
:1038E80039CEE49003F9F022EF640660030239CE82
:1038F800900405E0640670030239CE9003F2E044B8
:1039080020F022E49003F9F0900402E0FD2408F589
:1039180082E43404F583E0FE74072DF582E4340470
:10392800F583E07C002400FFEC3EFE9003FCE06E93
:103938007003A3E06F60079003F2E04480F0900307
:10394800F2E0FF6006900406F08007D24CE4900491
:1039580006F0E4900402F0900405740BF090040360
:10396800E0FFA3E0900403F0A3EFF07F02900402CD
:10397800E0FE2407FDE433FCEFC39DEC6480F8749B
:103988008098501874002FF582E43404F583E0FD24
:103998009002B5E48DF01223C40F80D19002B5E0F7
:1039A800FCA3E0FF74072EF582E43404F583EFF0FE
:1039B800ECFF900402E02408F582E43404F583EF78
:0639C800F0C29C75995A43
:0139CE0022D6
:105294009003F9E02400F582E43404F583EFF09000
:1052A40003F9E004F0E0C3948C4002E4F09003F9C5
:1052B400E064017027900400E0FF54FEB59A10EFFB
:1052C40020E006D246C2498013D249C246800D90DE
:1052D4000400E0645A6005E49003F9F030460D9050
:1052E40003F9E0640370301239CF802B30492590E4
:1052F4000402E02403FFE433FE9003F9E0D39FEEBD
:105304006480F8748098400F12500EC249E49003F0
:10531400F9F08003123868C243E49005E8F0900580
:07532400E9F09003F6F0220E
:104EB800900400E0B45A06A3E064A56003304C44B3
:104EC800900402E02408FFE433FE9003F9E0C39F56
:104ED800EE6480F87480984014D29CE4F0C2469046
:104EE8000400F0A3F0A3F0A3F0D24380609003F98C
:104EF800E004F0C29CE02400F582E43404F583E089
:104F0800F59980499003F9E0FF6016900402E024C7
:104F180003FDE433FCC3EF9DEC6480F87480984093
:104F280017D29CE49003F9F0C246900400F0A3F075
:104F3800A3F0A3F0D24380159003F9E004F0C29CDB
:104F4800E02400F582E43404F583E0F599E4900563
:0B4F5800E8F09005E9F09003F6F0226D
:107282009003F6E004F0C394044008E4F09003F99C
:04729200F0D29C2278
:1071F800305C119002B1E004F0C39405400BD25A00
:0A7208007405F022E49002B1F022B8
:0E4F63009002C0EFF0A3EDF0A3EAF0A3EBF094
:104F7100C254E4A3F0305A03025006A3F09002C1D8
:104F8100E0FF9002C5E0C39F507B9002C4E0FF04A4
:104F9100F0EFC39405503E9002C0E0FD7C0090020A
:104FA100F97401F0A3F09002C2E0FFA3E09002FBCC
:104FB100CFF0A3EFF0E4FB7F36123B1F9254305445
:104FC10004801280C5E4F5C87F0112689012724115
:104FD10012689080B59002C4E0C394054004802516
:104FE1008015E49002C4F09002C0E004F09002C287
:104FF100E475F0011223C47F011268909002C5E0AC
:0C50010004F0024F7EA254B3925CA25453
:01500D002280
:0E5B8B009002C3EFF0A3EDF0A3EAF0A3EBF05D
:105B9900C254E4A3F0205A4D9002C7E0FF04F0EF8D
:105BA900C3940550409002C3E0FD7C00A3E090023D
:105BB900EFF0A37401F09002C5E0FFA3E09002F1B9
:105BC900CFF0A3EFF0E4FB7F361230A492543054A7
:105BD90004801280C3E4F5C87F01126890127241F3
:0C5BE90012689080B3A254B3925CA254E6
:015BF500228D
:106D06007A027BA37D02E4FF125B8B502E9002A3D6
:106D1600E07004A3E060249002A7E04480F07A02C9
:106D26007BA77D017F04124F639002A7E0547FF09A
:0C6D36007A027BA77D017F04124F6322CC
:1055F000E49002A6F0A37450F0E4A3F0A374F8F0D2
:10560000E4A3F0A3F0A37470F0A37401F0A37403F7
:10561000F0A374FFF0E4A3F03000199002A7E04477
:1056200008F09002ACE0FF9000BBE0540FFEEF4E9C
:105630009002ACF030013E9002A7E04404F09002EA
:10564000ADE0FF9000BBE054F0FEEF4E9002ADF0F5
:105650009000BCE0FEA3E0FF7C007D32122688E4CF
:105660007B257A01F9F8122480AD07AC06EC900294
:05567000AEF0A3EFF015
:015675002212
:10556900D2539002BF7403F09002BFE0FF14F0EF32
:1055790060727A027BA67D0B7F03124F63505C90A9
:1055890002BE7403F09002BEE0FFD3940B504E7A32
:10559900027BBC7D02125B8B9002BEE0FF7E007B2A
:1055A9000124A3F9EE3402FA122344FD9002BCE06F
:1055B900B5051374A42FF9EE3402FA122344FF90AF
:1055C90002BDE06F600C9002BEE064076004C25344
:1055D900800B9002BEE02402F080AAC253305388A7
:0655E90080028084A25341
:0155EF002299
:106CC9007A027BA37D02E4FF125B8B502F9002A412
:106CD900E0FF30E102D259EF30E002D25B9002A32B
:106CE900E0FF30E307206804D215D26AEF30E202F0
:0D6CF900D2149002A4E030E203125569228B
:107212007A027BB97D027F02125B8B500A9002B91F
:07722200E09002A5F0F52643
:017229002242
:105DF9009002BB7403F09002BBE0FFD3940B5050A8
:105E09007A027BB97D02125B8B9002BBE0FF7E00B8
:105E19007B0124A3F9EE3402FA122344FD9002B95E
:105E2900E0B5051374A42FF9EE3402FA122344FFE6
:105E39009002BAE06F60109002BBE064076008123C
:105E49005569400CD263229002BBE02402F080A67F
:015E59002226
:107057009002B07433F07A027BB07D017F0D124F3E
:107067006350129002A7E04420F07A027BA77D01CB
:067077007F04124F6322AA
:107258009002A8E054FCF04FF07A027BA87D017FF1
:0572680005124F632236
:1072BD009002A7E04401F07A027BA77D017F0412C2
:0372CD004F6322EA
:1072D0009002A7E054FEF07A027BA77D017F0412A2
:0372E0004F6322D7
:1072E3009002A7E04402F07A027BA77D017F04129B
:0372F3004F6322C4
:1072F6009002A7E054FDF07A027BA77D017F04127D
:037306004F6322B0
:106C8A009002BBEEF0A3EFF09002BBE0FEA3E07827
:106C9A0005CEC313CE13D8F99002AAF07A027BAAC2
:106CAA007D017F07124F6350159002BBE0A3E0906D
:0F6CBA0002ABF07A027BAB7D017F08124F6322A1
:107309009002A7E04410F07A027BA77D017F041266
:037319004F63229D
:10731C009002A7E054EFF07A027BA77D017F041264
:03732C004F63228A
:10732F009002A9E044F8F07A027BA97D017F061252
:03733F004F632277
:107342009002A9E05407F07A027BA97D017F061220
:037352004F632264
:107355009002A9E044E0F07A027BA97D017F061244
:037365004F632251
:107368009002A9E0541FF07A027BA97D017F0612E2
:037378004F63223E
:10737B009002A9E04408F07A027BA97D017F0612F6
:03738B004F63222B
:10738E009002A9E054F7F07A027BA97D017F0612E4
:03739E004F632218
:1073B3009002A6E04FF07A027BA67D017F03124F75
:0273C300632243
:10722A009002A6E0FEEFF4FFEE5FF07A027BA67D05
:07723A00017F03124F6322E4
:103C6600305E03023DA9305F03023DA92003030233
:103C76003DA9E490053AF0A3F0C3900063E09512E5
:103C8600900062E09511500330181ED3900065E055
:103C96009512900064E09511400320180C2010093D
:103CA600201206201103301308C260E4900539F093
:103CB60022C39000A3E095129000A2E09511400364
:103CC600023DA2C3E5129510FFE511950FFED390B4
:103CD60000A5E09F9000A4E09E4003023DA2900054
:103CE600A6E0FEA3E0FFEE3395E0FDFC9002201275
:103CF60025B3C312252D5003023DA2206006900570
:103D060039E004F09000A8E075F00AA4FF900539A8
:103D1600E0C39FE5F06480F87480985003023DA9E3
:103D2600AD14E5142513FFE433FEEDC39FEE648066
:103D3600F87480985063ED25E0240AF582E4340295
:103D4600F583E0FEA3E0C39510FFEE950FFED3903A
:103D560000A5E09F9000A4E09E503BED25E0240ADC
:103D6600F582E43402F583E0FEA3E0FF9000A2E0D2
:103D7600FAA3E0FBC3EF9BEE9A401B74017E00A8FA
:103D860005088005C333CE33CED8F9FF90053AE057
:103D96004EF0A3E04FF00D8089D26022C260E4901D
:033DA6000539F0EC
:013DA90022F7
:106E2500C25330052D20162A306227C39002B4E0E4
:106E350094B49002B3E094005011D253900538E019
:106E450004F0C3940A400BD2168007C262E4900591
:046E550038F0A2531C
:016E59002216
:104BF200C3E5129510FFE511950FFEC3EF94B0EED9
:104C02009404500AE5129464E51194055002D262AC
:104C1200900536E024FE605514605914606A1460F1
:104C22007C24046003024CAB205F0330607B306164
:104C32001590053AE05455FFA3E054559002B9CFC0
:104C4200F0A3EFF0801390053AE054AAFFA3E054DA
:104C5200AA9002B9CFF0A3EFF09002B9E0FEA3E070
:104C6200FF126C8A9005367402F0D25E22900536ED
:104C72007403F022126E254030E4FFFE126C8A901B
:104C820005367404F0B26122126E25400790053693
:104C92007405F0229005367401F0B2612290053657
:094CA2007401F0C25FC260C25E41
:014CAB0022E6
:10707D0030052220161F900537E004F0C3942D40F3
:10708D0014742DF0205E0EE4F0D25F90053A740377
:06709D00F0A374FFF022D5
:0A73ED00123C6612707D124BF22272
:106EC400FFD8FFE2FFECFFF60000000A00190023E0
:106ED400002D00370041004B0055FFFBFFFCFFFD78
:106EE400FFFEFFFFFFFF000000010001000200039E
:046EF4000004000591
:042B2D008F828E8382
:102B31007E037FE8AD82AC83122688C006C007AE53
:102B410083AF82C3E49FFF74109EFEAB07FAE4F9E2
:102B5100F8D007D0061224809002BC122600E47F30
:102B61000AFEFDFC9002BC1225B3D3122543401D81
:102B71009002BC12259AC3EF940AFFEE9400FEED79
:102B81009400FDEC9400FC9002BC122600903DAA3A
:102B9100E493FE740193FFE4FCFD9002BC1225B3A3
:102BA100C3122543400D9002BA7408F0A374B7F024
:102BB100022D14903EEAE493FE740193FFE4FCFDC0
:102BC1009002BC1225B3D3122543500D9002BA7462
:102BD1000EF0A374F7F0022D1490027CE09002B97C
:102BE100F075F002903DAA122656E493FE7401930B
:102BF100FFE4FCFD9002BC1225B3D3122543403BF8
:102C010090027CE0149002B9F09002B9E0FFC39405
:102C110000406975F002EF903DAA122656E493FE3A
:102C2100740193FFE4FCFD9002BC1225B3D312257D
:102C31004340499002B9E014F080CE90027CE00458
:102C41009002B9F09002B9E0FFC394A0502875F04A
:102C510002EF903DAA122656E493FE740193FFE41D
:102C6100FCFD9002BC1225B3D312254350089002FB
:102C7100B9E004F080CE9002B9E014F09002B9E01E
:102C810090027CF075F002903DAA122656E493FE64
:102C9100740193FFE4FCFD9002BC1225B31223E7FB
:102CA100E47B0AFAF9F81223F5C004C005C006C096
:102CB100079002B9E0FF75F002903DAC122656E490
:102CC10093FC740193FD75F002EF903DAA12265614
:102CD100C37401939DFFE4939CFEAB07FAE4F9F8FA
:102CE100D007D006D005D004122480AB07AA0690E5
:102CF100027CE024CEFFE434FFFE7C007D0A122337
:102D01005DEF2BFFEE3ACF24ABCF340A9002BAF03D
:0B2D1100A3EFF09002BAE0FEA3E0FF89
:012D1C002294
:10669100D2539002C2E514F0E5132514FFE433FE52
:1066A1009002C2E0C39FEE6480F87480985028E0A5
:1066B100FF25E02485F582E43402AB82FAEF25E080
:1066C100240EFF7D02125B8B4005C253A253229020
:0966D10002C2E004F080C1A253F2
:0166DA00229D
:10684800D2537A027B997D027F22125B8B4002C26F
:10685800537A027B9B7D027F24125B8B4002C253DA
:106868007A027B9D7D027F26125B8B4002C253E534
:1068780013D39405400F7A027B9F7D027F28125B19
:076888008B4002C253A25332
:01688F0022E6
:10437C001268484003024459900299E0FEA3E0FF02
:10438C00122B2D9000C6E02FFF9000C5E03EFEC220
:10439C00AC900224F0A3EFF0D2AC90029DE0FEA30F
:1043AC00E0FF7C007D11122688E47B0AFAF9F812F2
:1043BC002480EF241FFFE43EFEC2AC900228F0A341
:1043CC00EFF0D2ACE513D39405402A90029FE0FEA7
:1043DC00A3E0FF7C007D11122688E47B0AFAF9F831
:1043EC00122480EF241FFFE43EFEC2AC90022AF0A0
:1043FC00A3EFF0D2AC900224E0FCA3E0FD9002020B
:10440C00ECF0A3EDF0900204ECF0A3EDF0300D3DD8
:10441C0090029BE0FEA3E0FF122B2D9000C8E02F32
:10442C00FF9000C7E03EFEC2AC900226F0A3EFF076
:10443C00D2ACD3900203E09F900202E09E4006EEC5
:0D444C00F0A3EFF022900204EEF0A3EFF0D9
:014459002240
:104025009002BA122625000000009002BE12262535
:1040350000000000E4900200F0A3F09002B37417B2
:10404500F0A37470F0126691400302415C9002B9CE
:10405500E514F0E5132514FFE433FE9002B9E0FD05
:10406500C39FEE6480F87480984003024133ED25C8
:10407500E02485F582E43402F583E0FEA3E0FF7CCD
:104085000E7DD8122688C006C0079000BFE0FEA3AB
:10409500E0FFFBAA06E4F9F8D007D00612248090C9
:1040A50002BE122600900200E0FEA3E0FFE4FCFD44
:1040B5009002BE1225B3D3122543400E9002BE12C4
:1040C500259A900200EEF0A3EFF09002B3E0FEA374
:1040D500E0FFE4FCFD9002BE1225B3C31225435058
:1040E5000E9002BE12259A9002B3EEF0A3EFF020D7
:1040F5005E33C2AC9002BE12259A9002B9E025E06B
:10410500240AF582E43402F583EEF0A3EFF0D2AC95
:104115009002BA12259A9002BE1225B31223DA90A4
:1041250002BA1226009002B9E004F0024058205E5F
:1041350026900200E0F511A3E0F5129002B3E0F538
:104145000FA3E0F510C2AC9002BA12259A90021E98
:07415500EEF0A3EFF0D2AC85
:01415C002240
:104CAC00E49002BEF0A3F0A3F09002C0E0FFC39426
:104CBC000C4003024D56EF25E024C4F582E4346E1B
:104CCC00F583E493FE740193FFFBAA06EA3395E0A7
:104CDC00F9F89002C0E025E024C6F582E4346EF5C4
:104CEC0083E493FE740193FFEE3395E0FDFC1223F5
:104CFC00DAE47B02FAF9F8126AC1E47B0AFAF9F8F1
:104D0C001223F5EF24ABFBEE340AFAE43DF9E43C54
:104D1C00F8900228E0FEA3E0FFE4FCFDC312252D71
:104D2C00401F9002C0E025E024DEF582E4346EF5ED
:104D3C0083E493FF7401939002BECFF0A3EFF08055
:104D4C00099002C0E004F0024CB59002BEE0FEA354
:024D5C00E0FF76
:014D5E002232
:103410009002BA122625000000007A027BA17D02EC
:103420007F2A125B8B9002A1E0FEA3E0FFEE30E466
:103430000944E09002A1F0A3EFF0124CAC9000C35D
:10344000E0FCA3E0FDC39002A2E09DFD9002A1E09C
:103450009CCD2FFFED3EFE3395E0FDFC7B187AFC02
:1034600079FF78FF1223F5C006C0079000C1E0FE87
:10347000A3E0FFFBAA06EA3395E0F9F8D007D006EF
:10348000126AC190027D12260090027D12259A9048
:1034900002B2E025E025E0243CF582E43402F58325
:1034A0001226009002B2E004F0C394104002E4F04F
:1034B000E49002B9F09002B9E0FFC394105026A343
:1034C0001225B3EF25E025E0243CF582E43402F533
:1034D0008312259A1223DA9002BA1226009002B9BA
:1034E000E004F080D0E47B10FAF9F89002BA1225DB
:1034F0009A126AC1900281122600C22BC22A900041
:1035000028E0FEA3E0FFC3E49FFFE49EFE3395E0C6
:10351000FDFC9002811225B3C312252D5021900489
:103520009FE004F0C3940A4067740AF0D22BC2AC47
:1035300090028112259A900220122600D2AC22908D
:103540000028E0FEA3E0FFEE3395E0FDFC90028151
:103550001225B3D312252D402990049EE004F09447
:103560000A402D740AF0D22A7D647FA07E0F125784
:1035700078C2AC90028112259A900220122600D2C5
:10358000AC22C2AC90022012262500000000D2AC72
:013590002218
:10729600126CC9C25B12402512437C305905C25993
:0472A600123410226C
:105AB200E49002B9F0A3F0AF14E513FDE5142DFD57
:105AC200E433FCEFC39DEC6480F8748098501DEFC2
:105AD20025E02485F582E43402F583E0FCA3E0FDB1
:105AE2009002B9EC8DF01223C40F80CD9002B9E080
:105AF200FEA3E0FF7C0E7DD8122688C006C0079068
:105B020005DFE0FEA3E0FFFBAA06E4F9F8D007D028
:0C5B1200061224809000BFEEF0A3EFF01C
:015B1E002264
:106D42009000C3E0FEA3E0FFC39002A2E09FFF9089
:106D520002A1E09EFE3395E0FDFC7B187AFC79FFF0
:106D620078FF1223F59005D61225B3126AC1EF4EB1
:0A6D720060089000C1EEF0A3EFF0FE
:016D7C0022F4
:1073C5009002A1E0FFA3E09000C3CFF0A3EFF0226D
:1069F300900299E0FEA3E0FF122B2DC39005DCE08B
:106A03009FFF9005DBE09EFE9000C5E0FCA3E0FD48
:106A1300C3EF9DFDEE9CFCC3ED9496EC64809480E3
:106A23005012ED946AEC6480947F40089000C5EEA8
:046A3300F0A3EFF0ED
:016A3700223C
:106A380090029BE0FEA3E0FF122B2DC39005DEE041
:106A48009FFF9005DDE09EFE9000C7E0FCA3E0FDFF
:106A5800C3EF9DFDEE9CFCC3ED9496EC648094809E
:106A68005012ED946AEC6480947F40089000C7EE61
:046A7800F0A3EFF0A8
:016A7C0022F7
:106A7D009005E1E0900497F09005E2E0900498F025
:106A8D009005E3E0900499F09005E4E090049AF00D
:106A9D009005E5E090049BF09005E6E090049CF0F5
:106AAD009005E7E090049DF07E047F971251F8D297
:046ABD003AD23D226A
:1063880030794BC2799005DAE030E003125AB290C6
:1063980005DAE030E403126D429005DAE030E503F7
:1063A8001273C59005DAE030E2031269F39005DA5A
:1063B800E030E303126A389005DAE030E703126A46
:0F63C8007DE49005DAF0D2709005F37402F022B4
:10651300306A0DC26AD268E49005F2F01272E32287
:1065230030683A127212203134900087E075F0021D
:10653300A4FFAEF09005F2E004F0C39FEE6480F890
:106543007480984018C268E4F01272F6307602C282
:0E65530019C21BC21C301505C215126D06229E
:1067B70030690DC269D267E49005F1F01272BD220B
:1067C70030673512721220302F900087E075F00283
:1067D700A4FFAEF09005F1E004F0C39FEE6480F8EB
:1067E7007480984013C267E4F01272D0307507C204
:0967F70018C214126D06C21A2228
:10716900300719303B119003E6E004F0C394054061
:0D7179000BD2397405F022E49003E6F022F9
:105E5A009002E3EEF0A3EFF0A3EDF0A3EAF0A3EBD8
:015E6A00F047
:105E6B00C253203941E4A3F09002E3E0FCA3E0FD30
:105E7B00A3E09002F9F0E4A3F09002E6E0FFA3E0C8
:105E8B009002FBCFF0A3EFF07B017FA0123B1F50E2
:105E9B0004D25380117F011268909002E8E004F065
:0D5EAB00E0C3940540C2A253B3923BA25342
:015EB80022C7
:105EB9009002C5EEF0A3EFF0A3EDF0A3EAF0A3EB97
:015EC900F0E8
:105ECA00C254203941E4A3F09002C5E0FCA3E0FDEE
:105EDA00A3E09002EFF0E4A3F09002C8E0FFA3E091
:105EEA009002F1CFF0A3EFF07B017FA01230A45013
:105EFA0004D25480117F011268909002CAE004F023
:0D5F0A00E0C3940540C2A254B3923BA254E0
:015F17002267
:105B1F007E027FBC7B08E4FD126FDFE49002BAF0D7
:105B2F00A3F09002BAE0FEA3E0FFE4FCFD7BFF7A56
:105B3F0007F9F8D312252D402E53B1F89002BAE091
:105B4F00FEA3E07805C333CE33CED8F9241FFFE48C
:105B5F003EFE7A027BBC7D01125E5A9002BAE4755A
:105B6F00F0011223C480BB7A027BBC7D087FE07EEC
:0B5B7F00FF125E5AE49003DFF0A3F079
:015B8A0022F8
:1057F900C2537A027BB97D087FE07EFF125EB992BF
:10580900539002BAE0FF9002B9E02F9002BBF090EA
:1058190002BEE0FF9002BDE02F9002BFF09002BCF3
:10582900E0FF9002BBE0B507179002B9E0FEA3E0E4
:105839007C002400FFEC3E9003DFF0A3EFF0802A08
:105849009002C0E0FF9002BFE0B507179002BDE0EB
:10585900FEA3E07C002400FFEC3E9003DFF0A3EF01
:0C586900F08007E49003DFF0A3F0A253EE
:015875002210
:1065AD00E49002C3F07E047F97122EE27E047F9763
:1065BD007C027DBA7B07126EF8E4FF74BA2FF58268
:1065CD00E43402F583E0FE9002C3E02EF00FEFB449
:1065DD0007E99002C3E09002C1F0A3745AF07A0269
:0B65ED007BBA7D097FF07EFF125E5A32
:0165F8002280
:106B8A009003DFE0FCA3E0FDEC9002DBF0AF05A38D
:106B9A00EFF09002DBE02F9002DEF09002DBE09053
:106BAA0002DFF09002DCE09002E0F09002DEE0907A
:106BBA0002E2F07A027BDB7D087FE07EFF125E5AFA
:016BCA0022A8
:05325D009002BAEFF041
:103262006410701A7E037FE77C027DBB7B03126EC3
:10327200F87E037FEB7C027DBE126EF8801F7E0417
:103282007F97122EE27E047F977C027DBB7B031226
:103292006EF87E047F9A7C027DBE126EF890020662
:1032A200E0FCA3E0FDEC9002C1F0A3EDF090020877
:1032B200E0FCA3E0FDEC9002C3F0A3EDF090022C41
:1032C20012259A78181225549002C5EFF090022C1C
:1032D20012259A78101225549002C6EFF090022C13
:1032E20012259A78081225549002C7EFF090022C0A
:1032F20012259A9002C8EFF090023012259A78189F
:103302001225549002C9EFF090023012259A7810DB
:103312001225549002CAEFF090023012259A7808D2
:103322001225549002CBEFF090023012259A9002AF
:10333200CCEFF090021EE0FCA3E0FDAE047818CEC4
:10334200C313CE13D8F99002CDF0EDAE047810CEAF
:10335200C313CE13D8F99002CEF090021EE0FCA364
:10336200E0FDEC9002CFF0A3EDF090022012259A3E
:1033720078181225679002D1EFF090022012259A58
:1033820078101225679002D2EFF090022012259A4F
:1033920078081225679002D3EFF090022012259A46
:1033A2009002D4EFF0900224E0FCA3E0FDEC900246
:1033B200D5F0A3EDF0900236E0FCA3E0FDEC900224
:1033C200D7F0A3EDF09002BAE09002D9F0A3745ABC
:1033D200F09003DFE0FEA3E0FF7A027BBB7D2012C8
:1033E2005E5A9003DFE475F0201223C49003DFE0FD
:1033F200FEA3E0FFE4FCFD7BE07AFFF9F8D312259F
:0D3402002D5007E49003DFF0A3F0126B8A59
:01340F00229A
:105C61009003F1E02480FFE434FFEF7D00C454F0A1
:105C7100FC900401E02488FFE434FFFEEF7807C3C1
:105C810033CE33CED8F92DFFEE3CFE900402E0FD79
:105C91007A047B03125EB97B017A047900900402D5
:105CA100E02403FD1271C0900402E02403F582E4B4
:105CB1003404F583EFF0C29C9003F9E02400F582EF
:085CC100E43404F583E0F599D9
:015CC90022B8
:1059D4009003F1E02480FFE434FFEF7D00C454F031
:1059E400FC9004A1E02488FFE434FFFEEF7807C3B1
:1059F40033CE33CED8F92DFFEE3CFE9004A2E0FD69
:105A04007A047BA3125EB97B017A0479A09004A284
:105A1400E02403FD1271C09004A2E024A3F582E403
:105A24003404F583EFF0758640C2A49003FAE024B1
:0E5A3400A0F582E43404F583E0F5A1E4F586E4
:015A42002241
:105A43009003F1E02480FFE434FFEF7D00C454F0C1
:105A5300FC900541E02488FFE434FFFEEF7807C3A0
:105A630033CE33CED8F92DFFEE3CFE900542E0FD58
:105A73007A057B43125EB97B017A05794090054232
:105A8300E02403FD1271C0900542E02443F582E453
:105A93003405F583EFF0758640C2949003FBE02450
:0E5AA30040F582E43405F583E0F591E4F586E4
:015AB10022D2
:106968007E047F97122EE27E047F977C047D037B52
:1069780007126EF87B017A047900900402E0240380
:10698800FD1271C0900402E02403F582E43404F59A
:1069980083EFF0C29C9003F9E02400F582E434040C
:0669A800F583E0F59922E1
:1065F9007E047F97122EE27E047F977C047DA37B25
:1066090007126EF87B017A0479A09004A2E02403B2
:10661900FD1271C09004A2E024A3F582E43404F5CC
:1066290083EFF0758640C2A49003FAE024A0F582B6
:0C663900E43404F583E0F5A1E4F58622CA
:106645007E047F97122EE27E047F977C057D437B37
:1066550007126EF87B017A057940900542E0240324
:10666500FD1271C0900542E02443F582E43405F53E
:1066750083EFF0758640C2949003FBE02440F582D9
:0C668500E43405F583E0F591E4F586228D
:104E0C00200703024EB7203A03024EB7C23A30389D
:104E1C0005C238125B1F9003E1E0FF7008A3E0703D
:104E2C0004A3E06021EF6008E49003E1F0125C6100
:104E3C009003E2E06005E4F0125A439003E3E06073
:104E4C0005E4F0125A439003EEE0FF7008A3E07003
:104E5C0004A3E06021EF6008E49003EEF0126968AF
:104E6C009003EFE06005E4F01265F99003F0E06068
:104E7C0005E4F0126645303D05C23D1265AD303C8F
:104E8C000CC23C9002B97410F0FF12325D30420C2F
:104E9C00C2429002B97401F0FF12325D303F0CC275
:0B4EAC003F9002B97402F0FF12325D6B
:014EB70022D8
:1045310020070302460390002EE0FF9003DCE00415
:10454100F0C39F4009E4F07E047F97122EE29003AE
:10455100DDE475F0011223C4FEC3E5F09410EE947E
:104561000E400BE49003DDF0A3F0D23AD23D202AB5
:104571001ED241304006C240D23AD24230190B30ED
:104581003E08C23ED23AD23F8005201902D23E30C7
:10459100416990002CE0FEA3E0FFEE3395E0FDFCC5
:1045A1009002201225B3C312252D404F9003E4E061
:1045B1007002A3E070147E047F97122EE27E047FC6
:1045C100977C037DE77B07126EF890002BE0FF7E5E
:1045D100007C007D3C12235D9003E4E475F0011240
:1045E10023C4FCD3E5F09FEC9E4017E49003E4F074
:1045F100A3F0D240C241D23AD23C22E49003E4F08B
:03460100A3F02201
:03105300025BF647
:105BF600C0E0C0D075D000C006C007C0867586005C
:105C060030D807C2D87F0112102E30D907C2D97FEB
:105C16000212102E30DA07C2DA7F0412102E30DBA1
:105C260007C2DB7F0812102E30DC07C2DC7F1012A1
:105C3600102E30DD07C2DD7F2012102E30DE07C2A7
:105C4600DE7F4012102E30DF07C2DF7F8012102E5B
:0B5C5600D086D007D006D0D0D0E032BE
:03102B00021003AD
:10100300C0E0C083C082C0D0C086758640C28F75E1
:1010130086001270C9D086D0D0D082D083D0E0327F
:1050B500307A0302515675090F20A705750901803D
:1050C5000620B003750902E509650C6038050EE593
:1050D5000E7002050DC3E50B940AE50A94004065C0
:1050E500E50E940AE50D94004067E50B9490E50AFA
:1050F50094014008E50C4440F5088003850C08D26E
:105105007A80428040E509640F6037E4F50DF50EBD
:10511500050BE50B7002050AB4900EE50AB401090A
:10512500E50C4410F508D27A22E50BB4B023E50A64
:10513500B4041E750A01750B90E50C4420F508D2E0
:105145007A2275080FE4F50AF50BF50DF50E8509BC
:015155000C4D
:015156002236
:106E5A00AB07AA06C2AF43A701EAF5F7AF038FFB58
:106E6A00AF058FFC75F26E75F30575F40A75F509B1
:106E7A00EAADF7B50509E475F6060000000000530F
:056E8A00A7FED2AF22BB
:1070A300D256E4FDFCEF2DFBEE3C8B82F583E4939B
:1070B3006004C256800D0DBD00010CE4B505E6EC7D
:0570C300B402E2A25638
:0170C80022A5
:08608A009002BFEEF0A3EFF05D
:10609200D256AE04AF05E4A3F0A3F09002C1E0FC37
:1060A200A3E0FDC3EC940250369002C0E02DFD90B7
:1060B20002BFE03C8D82F583E493FD9002C1E0FAD9
:1060C200A3E02FF582EE3AF583E0FCED6C6004C2AA
:1060D20056800C9002C1E475F0011223C480BCA268
:0160E2005667
:0160E300229A
:0854DD009002BFEEF0A3EFF016
:1054E500C256AF05A3ECF0A3EFF0E4FDFC9002BFBC
:1054F500E0FAA3E0FB2DF5FBEB2DEA3CF5F7A3E085
:10550500FEA3E02DF582EE3CF583E0F5FC75F26E29
:1055150020AF3D75F305E5A7603275F40A9005F4F3
:10552500E06455702375F5099002C0E02D9002BF27
:10553500E03CABF7B5030DE475F60600000000008E
:10554500D2568010C2568019C2568015C256801197
:10555500C256800D0DBD00010CED7003EC640270A8
:035565008CA256BF
:015568002220
:0E532B009002BBEEF0A3EFF0A3ECF0A3EDF0C8
:10533900C25553B1F8C2AF43A7019002BBE0FF7E4B
:1053490000F5F775F2E620AF5B75F305E5A7605444
:1053590075F40A9005F4E06455704975F509ADF7DF
:10536900EF6D7001EE703D75F606000000000090CB
:1053790002BBE0FEA3E0FF1270A350289002BBE03D
:10538900FEA3E0FFA3E0FCA3E0FD1254DD5015905D
:1053990002BBE0FEA3E0FFA3E0FCA3E0FD12608AEC
:1053A9005002D255E4F5F2F5F3F5F4F5F5F5F653B7
:0853B900A7FEF5F7D2AFA255E3
:0153C10022C9
:1046C800C253C254206F03024788C26F9005F47426
:1046D80055F0E513D39405400C9002B97427F0A364
:1046E8007410F0800A9002B97413F0A37488F090E3
:1046F80002B9E0FEA3E0FFC390021FE09F90021EF4
:10470800E09E406B9001FEE0645A7004A3E064A54B
:10471800705DFDFCFFFE12532B4023E4FDFCFFFE01
:1047280012532B4019D25374FF9001FEF0A3F0FDF1
:104738007FFE7E01126E5A7DFF7FFF126E5AE4FDE6
:10474800FCFF7E0212532B402AE4FDFCFF7E02127E
:10475800532B401FD25474FF9001FEF0A3F0FD7F4D
:10476800FE7E03126E5A7DFF7FFF126E5A8004D2BE
:1047780053D254E49005F4F0305305305402D26E0D
:01478800220E
:0E5F18009002B9EEF0A3EFF0A3EAF0A3EBF0D5
:105F2600D253AE04AF058E198F1AC2AF43A70153E1
:105F3600B1F8E4FFFED39002BCE09F9002BBE09E66
:105F460040279002BAE02FFD9002B9E03E8D82F51F
:105F560083E493851A82851983F0051AE51A70027F
:105F660005190FBF00010E80CC53A7FED2AFA25376
:015F76002208
:10726D003070119005F3E004F0C394024006C27033
:05727D00E4F0D26F22D5
:10700900C25343A701EEC313FEEF1325E0FFEE338E
:107019008F82F583740193B4A507E493B45A02D21D
:067029005353A7FEA25321
:01702F00223E
:0D3EEC009002BAECF0A3EDF09002B9EFF0F7
:103EF900758640EF64557051A3E0FEA3E0FFC394BB
:103F0900E8EE940350187588027C007D20122688FB
:103F1900C3E49FFFE49EA3F0A3EFF002401375886A
:103F2900229002BAE0FEA3E0FF7C007D20122688E1
:103F3900E47B40FAF9F8122480C3E49FFFE49E90E1
:103F490002BCF0A3EFF00240139002B9E0644470A0
:103F59005BA3E0FEA3E0FFC394A0EE940F5023758A
:103F690088127C007D80122688E47B08FAF9F81211
:103F79002480C3E49FFFE49E9002BCF0A3EFF0020B
:103F890040137588329002BAE0FEA3E0FF7C007D01
:103F990080122688E4FB7A01F9F8122480C3E49F91
:103FA900FFE49E9002BCF0A3EFF0805E9002B9E0BE
:103FB9007058A3E0FEA3E0FFC394F4EE94015022ED
:103FC9007588307C5D7DC0122688E4FB7A01F9F89A
:103FD900122480C3E49FFFE49E9002BCF0A3EFF09B
:103FE90080287588329002BAE0FEA3E0FF7C007D4C
:103FF90080122688E4FB7A01F9F8122480C3E49F31
:10400900FFE49E9002BCF0A3EFF09002BCE0FEA397
:0B401900E0F58CEEF58DD28AE4F58610
:014024002279
:10629500A2AFE433FEC2AFEF600D64206009EF6486
:1062A500406004EFB46007EF4408F5B28010EF6476
:1062B500806004EFB4A00753B2FB0053B2F70000AF
:1062C500000000000000EF600D64206009EF6440ED
:1062D5006004EFB4600343B204AF06EE24FF92AF4F
:0162E5002296
:105676009005EBEEF0A3EFF0A3EDF075C7B0900543
:10568600EBE0FEA3E0FFFBAA06E4F9F87FD87EB8BC
:105696007D05FC126AC18FCC9005EBE0FEA3E0FF0E
:1056A600FBAA06E4F9F87FD87EB87D05FC126AC12C
:1056B60078081225678FCDAFCDEFFEADCC7C00E428
:1056C6002DFFEC3EFE9005EDE0FBFD12235D7D64B3
:1056D60012236F8FCEAFCDEFFEADCC7C00E42DFF55
:1056E600EC3EFEAD0312235D7D6412236FEEF5CF13
:0156F6002291
:1056F7009005EEEEF0A3EFF0A3EDF075B6B09005D0
:10570700EEE0FEA3E0FFFBAA06E4F9F87FD87EB837
:105717007D05FC126AC18FAE9005EEE0FEA3E0FFA7
:10572700FBAA06E4F9F87FD87EB87D05FC126AC1AA
:1057370078081225678FAFAFAFEFFEADAE7C00E400
:105747002DFFEC3EFE9005F0E0FBFD12235D7D642E
:1057570012236F8FA4AFAFEFFEADAE7C00E42DFF39
:10576700EC3EFEAD0312235D7D6412236FEEF5A5BB
:01577700220F
:105778009002BEEEF0A3EFF0A3EDF075B7B0900283
:10578800BEE0FEA3E0FFFBAA06E4F9F87FD87EB8E6
:105798007D05FC126AC18FBC9002BEE0FEA3E0FF4B
:1057A800FBAA06E4F9F87FD87EB87D05FC126AC129
:1057B80078081225678FBDAFBDEFFEADBC7C00E455
:1057C8002DFFEC3EFE9002C0E0FBFD12235D7D64E0
:1057D80012236F8FBEAFBDEFFEADBC7C00E42DFF82
:1057E800EC3EFEAD0312235D7D6412236FEEF5BF20
:0157F800228E
:10689000E5B2547070067C067D868020E5B25470A7
:1068A000FEBE20067C037D438012E5B25470FEBE1E
:1068B00040067C017DA180047C007D8BE4FEEEC35C
:1068C0009F5014E4FBFAC3EB9DEA9C50070BBB00FE
:0768D000010A80F20E80E7CF
:0168D700229E
:105D300090002FE0645A705A900061E0645A7052EB
:105D4000900073E0645A704A900088E0645A704290
:105D500090008DE0645A703A900098E0645A703276
:105D60009000A1E0645A702A9000A9E0B45A2390F0
:105D700000BAE0B45A1C9000BEE0B45A159000CAB4
:105D8000E0B45A0E9001FEE0645A7004A3E064A5EA
:065D90006002C322D322D1
:086FDF009002C5EEF0A3EFF0F3
:106FE700E4FFEFC39B501A9002C5E0F8A3E0F582D7
:106FF7008883EDF09002C5E475F0011223C40F8079
:01700700E1A7
:017008002265
:086EF8009002DBEEF0A3EFF0C5
:106F0000E4FFEFC39B50239002DBE0F8A3E0F5829F
:106F10008883E08D828C83F00DBD00010C9002DB34
:0A6F2000E475F0011223C40F80D8BD
:016F2A002244
:0C73D500758E5543870100000000002267
:0C73E100758E554387020000000000225A
:106F88009005EAE06412702320430620440330454C
:106F98001A207017206F14C2AFE4F5A8F5A9F58878
:0C6FA800F5E8F59DF59CF598120000221C
:1066DB00D228D229201403301602C22820110F20F1
:1066EB00130C201B09201C06201503301602C2298F
:1066FB00202B0E201009201206201803301A02C27C
:10670B0028202A05301902C229201B06201C033021
:0A671B001502C228301A02C229221A
:106F5B001266DBA273302801B34008A274302901FA
:106F6B00B35019A2289273A2299274A229E433FF79
:0D6F7B0025E0FFA228E4334FFF12725822D8
:1068D800201844C3900063E09512900062E095117F
:1068E800501F9003BEE475F0011223C4FEC3E5F007
:1068F8009401EE94004020D218E49003BEF0A3F077
:1069080022D3900065E09512900064E0951140074D
:08691800E49003BEF0A3F0229D
:10692000201944D3900075E09510900074E0950F05
:10693000401F9003C0E475F0011223C4FEC3E5F0CC
:106940009401EE94004020D219E49003C0F0A3F02B
:1069500022C3900077E09510900076E0950F5007E5
:08696000E49003C0F0A3F02253
:1063D70020104B90008EE0FEA3E0FF900204E0FC4B
:1063E700A3E0FDD39FEC9E401F9003D0E475F0011E
:1063F7001223C4FEC3E5F09401EE94004020D210AE
:10640700E49003D0F0A3F022900090E0FEA3E0FF19
:0F641700C3ED9FEC9E5007E49003D0F0A3F0225A
:1064260020124B900092E0FEA3E0FF900202E0FCF7
:10643600A3E0FDC39FEC9E501F9003D4E475F001CA
:106446001223C4FEC3E5F09401EE94004020D2125C
:10645600E49003D4F0A3F022900094E0FEA3E0FFC2
:0F646600D3ED9FEC9E4007E49003D4F0A3F02207
:1064750020114B900099E0FEA3E0FF900204E0FCA0
:10648500A3E0FDD39FEC9E401F9003D2E475F0017D
:106495001223C4FEC3E5F09401EE94004020D2110E
:1064A500E49003D2F0A3F02290009BE0FEA3E0FF6E
:0F64B500C3ED9FEC9E5007E49003D2F0A3F022BA
:1064C40020134B90009DE0FEA3E0FF900202E0FC4D
:1064D400A3E0FDC39FEC9E501F9003D6E475F0012A
:1064E4001223C4FEC3E5F09401EE94004020D213BD
:1064F400E49003D6F0A3F02290009FE0FEA3E0FF17
:0F650400D3ED9FEC9E4007E49003D6F0A3F02266
:106D7D00307B3712402512437C1268D812692012DD
:106D8D0063D71264261264751264C49005F7E0048B
:106D9D00F0C394024014C27B205A09203906207892
:0B6DAD0003306E03D263221237002275
:1046040020185C201459C3900063E0951290006256
:10461400E095115033900066E075F00AA4FFAEF007
:104624009003BEE475F0011223C4FCC3E5F09FECD3
:104634009E50030246C7D218C275E49003BEF0A38D
:10464400F09003D8F0A3F022D3900065E095129087
:104654000064E09511406CE49003BEF0A3F02220C6
:104664007561D3900065E09512900064E095114067
:104674003C900067E075F00AA4FFAEF09003D8E424
:1046840075F0011223C4FCC3E5F09FEC9E40343066
:104694000E06D275D2698007C218C214126D06E4E0
:1046A4009003BEF0A3F09003D8F0A3F022C39000CF
:1046B40063E09512900062E095115007E49003D8EE
:0446C400F0A3F0224D
:10484600201959D3900075E09510900074E0950FEB
:104856004033900078E075F00AA4FFAEF09003C0F4
:10486600E475F0011223C4FCC3E5F09FEC9E5003EF
:10487600024901D219C276E49003C0F0A3F0900376
:10488600DAF0A3F022C3900077E09510900076E06E
:10489600950F5067E49003C0F0A3F02220765CC326
:1048A600900077E09510900076E0950F50379000D5
:1048B60079E075F00AA4FFAEF09003DAE475F00132
:1048C6001223C4FCC3E5F09FEC9E402F300F06D2A6
:1048D60076D26A8002C219E49003C0F0A3F0900376
:1048E600DAF0A3F022D3900075E09510900074E002
:0C48F600950F4007E49003DAF0A3F022D5
:1049020020105E90008EE0FEA3E0FF900204E0FC27
:10491200A3E0FDD39FEC9E4031900096E075F01429
:10492200A4FFAEF09003D0E475F0011223C4FAC3E1
:10493200E5F09FEA9E50030249BDD210E49003D0F5
:10494200F0A3F09003C2F0A3F022900090E0FEA347
:10495200E0FFC3ED9FEC9E5062E49003D0F0A3F021
:1049620022900090E0FEA3E0FF900204E0FCA3E0AE
:10497200FDC39FEC9E502E900096E075F014A4FFAC
:10498200AEF09003C2E475F0011223C4FAC3E5F05D
:104992009FEA9E4026C210E49003D0F0A3F0900359
:1049A200C2F0A3F02290008EE0FEA3E0FFD3ED9FC1
:0C49B200EC9E4007E49003C2F0A3F0224A
:1049BE0020125E900092E0FEA3E0FF900202E0FC67
:1049CE00A3E0FDC39FEC9E5031900096E075F0146D
:1049DE00A4FFAEF09003D4E475F0011223C4FAC321
:1049EE00E5F09FEA9E5003024A79D212E49003D476
:1049FE00F0A3F09003C6F0A3F022900094E0FEA383
:104A0E00E0FFD3ED9FEC9E4062E49003D4F0A3F060
:104A1E0022900094E0FEA3E0FF900202E0FCA3E0EF
:104A2E00FDD39FEC9E402E900096E075F014A4FFEF
:104A3E00AEF09003C6E475F0011223C4FAC3E5F09C
:104A4E009FEA9E4026C212E49003D4F0A3F0900396
:104A5E00C6F0A3F022900092E0FEA3E0FFC3ED9F0C
:0C4A6E00EC9E5007E49003C6F0A3F02279
:104A7A0020115E900099E0FEA3E0FF900204E0FCA2
:104A8A00A3E0FDD39FEC9E4031900096E075F014B0
:104A9A00A4FFAEF09003D2E475F0011223C4FAC366
:104AAA00E5F09FEA9E5003024B35D211E49003D2FF
:104ABA00F0A3F09003C4F0A3F02290009BE0FEA3C1
:104ACA00E0FFC3ED9FEC9E5062E49003D2F0A3F0A6
:104ADA002290009BE0FEA3E0FF900204E0FCA3E02A
:104AEA00FDC39FEC9E502E900096E075F014A4FF33
:104AFA00AEF09003C4E475F0011223C4FAC3E5F0E2
:104B0A009FEA9E4026C211E49003D2F0A3F09003DC
:104B1A00C4F0A3F022900099E0FEA3E0FFD3ED9F3A
:0C4B2A00EC9E4007E49003C4F0A3F022CE
:104B360020135E90009DE0FEA3E0FF900202E0FCE1
:104B4600A3E0FDC39FEC9E5031900096E075F014F3
:104B5600A4FFAEF09003D6E475F0011223C4FAC3A5
:104B6600E5F09FEA9E5003024BF1D213E49003D680
:104B7600F0A3F09003C8F0A3F02290009FE0FEA3FC
:104B8600E0FFD3ED9FEC9E4062E49003D6F0A3F0E5
:104B96002290009FE0FEA3E0FF900202E0FCA3E06B
:104BA600FDD39FEC9E402E900096E075F014A4FF76
:104BB600AEF09003C8E475F0011223C4FAC3E5F021
:104BC6009FEA9E4026C213E49003D6F0A3F090031A
:104BD600C8F0A3F02290009DE0FEA3E0FFC3ED9F86
:0C4BE600EC9E5007E49003C8F0A3F022FE
:1060E400201A5590006D12259A90027D1225B3D383
:1060F40012252D402A900071E075F00AA4FFAEF03D
:106104009003CCE475F0011223C4FCC3E5F09FECCA
:106114009E4025D21AD269E49003CCF0A3F0222049
:106124006716D39003CDE094009003CCE094004034
:096134000774FFF5F01223C422E8
:10613D00201B5590007D12259A90027D1225B3C328
:10614D0012252D502A900081E075F00AA4FFAEF0C3
:10615D009003BAE475F0011223C4FCC3E5F09FEC83
:10616D009E4025E49003BAF0A3F0D21BD26A222000
:10617D006816D39003BBE094009003BAE0940040FE
:09618D000774FFF5F01223C4228F
:10619600201C5590008212259A90027D1225B3C3C9
:1061A60012252D502A900086E075F002A4FFAEF06D
:1061B6009003BCE475F0011223C4FCD3E5F09FEC18
:1061C6009E4025E49003BCF0A3F0D21CD26A2220A4
:1061D6006816D39003BDE094009003BCE0940040A1
:0961E6000774FFF5F01223C42236
:10712C00207B1B1246041248461249021249BE1219
:0F713C004A7A124B361260E412613D12619622BC
:1058EE00300272201B06201C03301539900072E026
:1058FE0075F014A4FFAEF09003CEE475F001122300
:10590E00C4FCC3E5F09FEC9E401BE49005F2F090C2
:10591E0003CEF0A3F0C21BC21CC26AC268301505CA
:10592E00C215126D06301A2D900072E075F014A497
:10593E00FFAEF09003CAE475F0011223C4FCD3E568
:10594E00F09FEC9E400FE49003CAF0A3F0C21A90B1
:06595E0005F1F0C2672212
:10718600300719307711900496E004F0C394054057
:0D7196000BD2787405F022E4900496F022EC
:0E5FD4009002F0EFF0A3EDF0A3EAF0A3EBF0E3
:105FE200C256207840E4A3F09002F0E0FD7C00A3CA
:105FF200E09002F9F0E4A3F09002F2E0FFA3E09057
:1060020002FBCFF0A3EFF0E4FB7FDE123B1F500454
:10601200D25680117F011268909002F4E004F0E001
:0C602200C3940540C3A256B39277A25667
:01602E00224F
:0E602F009002E6EFF0A3EDF0A3EAF0A3EBF091
:10603D00C255207840E4A3F09002E6E0FD7C00A379
:10604D00E09002EFF0E4A3F09002E8E0FFA3E0900F
:10605D0002F1CFF0A3EFF0E4FB7FDE1230A4500489
:10606D00D25580117F011268909002EAE004F0E0B1
:0C607D00C3940540C3A255B39277A2550E
:0160890022F4
:082EE2009002DBEEF0A3EFF01B
:102EEA00C2547A027BDD7D09E4FF12602F4003029F
:102EFA0030A19002E4E030E0030230949002DFE077
:102F0A0020E703022FB39002DDE0FF547094504093
:102F1A0003022FB3EF540F94094003022FB3E05476
:102F2A007F94594003022FB3A3E0FF54709450508A
:102F3A0078EF540F94095071E0547F9459506AA362
:102F4A00E0FF543094205061EF540F9409505AE036
:102F5A00542F94245053A3E0FF54309430504AEF36
:102F6A00540F94095043E0543FFF9431503BEF60B3
:102F7A0038A3E0FF54109410502FEF540F940950C7
:102F8A0028E0541FFF94125020EF601DA3E0FF5465
:102F9A00F094905014EF540F9409500DE094995006
:102FAA0008A3E05407940640779002DBE0FEA3E012
:102FBA00FFF5828E83E09002DDF08F828E83A3E09C
:102FCA009002DEF09002DBE0A3E0F5828E83A3A3F9
:102FDA00E09002DFF08F828E83A3A3A3E09002E049
:102FEA00F09002DBE0A3E02404F582E43EF583E0FE
:102FFA009002E1F0EF2405F582E43EF583E09002C9
:10300A00E2F09002DBE0A3E02406F582E43EF583D9
:10301A00E09002E3F07E027FDD1251F8925480774D
:10302A009002DDE0FF9002DBE0FCA3E0FDF5828C7C
:10303A0083EFF09002DEE08D828C83A3F09002DFB2
:10304A00E0541F8D828C83A3A3F09002E0E08D826E
:10305A008C83A3A3A3F09002E1E0FFED2404F582A0
:10306A00E43CF583EFF09002E2E0FFED2405F582FF
:10307A00E43CF583EFF09002E3E0FFED2406F582ED
:10308A00E43CF583EFF0D254800D9002DBE0FEA31E
:09309A00E0FF1251F89254A25417
:0130A300220A
:0851F8009002E6EEF0A3EFF0D7
:10520000C255A37490F07A027BE87D017F07125F9C
:10521000D492559002E6E0FEA3E0FFF5828E83E093
:105220009002E9F08F828E83A3E09002EAF0900270
:10523000E6E0FCA3E0FDF5828C83A3A3E04480902C
:1052400002EBF08D828C83A3A3A3E09002ECF0909C
:1052500002E6E0A3E0FF2404F582E43EF583E0905B
:1052600002EDF0EF2405F582E43EF583E09002EED6
:10527000F09002E6E0A3E02406F582E43EF583E048
:105280009002EFF07A027BE97D07E4FF125FD4928F
:0352900055A255CF
:0152930022F8
:085450009002B9EEF0A3EFF0A9
:10545800C253E49002C4F07E027FBB7B09FD126F49
:10546800DF7A027BBB7D097FF07EFF125EB9E4FF25
:1054780074BB2FF582E43402F583E0FE9002C4E0A9
:105488002EF00FEFB407E99002C4E0FF9002C2E0EB
:10549800B50706A3E0645A601BE49002BBF0A3F0D2
:1054A800A37412F0A37401F0A37405F0A37420F0A0
:1054B800A37405F07E027FBB9002B9E0FCA3E0FD77
:1054C8007B07126EF89002B9E0FEA3E0FF122EE20D
:0454D8009253A253F6
:0154DC0022AD
:10427C0000070E091C1B1215383F363124232A2D3A
:10428C0070777E796C6B6265484F464154535A5D2A
:10429C00E0E7EEE9FCFBF2F5D8DFD6D1C4C3CACD1A
:1042AC0090979E998C8B8285A8AFA6A1B4B3BABD0A
:1042BC00C7C0C9CEDBDCD5D2FFF8F1F6E3E4EDEAFA
:1042CC00B7B0B9BEABACA5A28F88818693949D9AEA
:1042DC002720292E3B3C35321F18111603040D0ADA
:1042EC005750595E4B4C45426F68616673747D7ACA
:1042FC00898E878095929B9CB1B6BFB8ADAAA3A4BA
:10430C00F9FEF7F0E5E2EBECC1C6CFC8DDDAD3D4A9
:10431C00696E676075727B7C51565F584D4A434499
:10432C00191E171005020B0C21262F283D3A333489
:10433C004E49404752555C5B7671787F6A6D646379
:10434C003E39303722252C2B0601080F1A1D141369
:10435C00AEA9A0A7B2B5BCBB9691989F8A8D848359
:10436C00DED9D0D7C2C5CCCBE6E1E8EFFAFDF4F349
:1071C000E4FFEDD3940040131223446F90427C936C
:0B71D000FF740129F9E43AFA1D80E782
:0171DB002291
:10703000D2587D807CBBE5C820E31053B1F8ED4CFD
:107040006009ED1D70011C80ED80EBE5D154F86FF7
:067050006002C258A258C4
:017056002217
:103B1F009002F8EBF09002F5EFF0A3ECF0A3EDF0CC
:103B2F00D25790030174BBF0A37480F09002FDEFA5
:103B3F00F0A3EDF09002FBE0FEA3E0F5828E83E0B0
:103B4F009002FFF07B017A0279FD7D031271C09024
:103B5F000300EFF09002F9E0D394005003023C63AE
:103B6F0043E6C043D10143C80175C8607F08127096
:103B7F0030400C7F101270304005C257023C40900D
:103B8F0002F5E0F58D75C8407F181270304005C200
:103B9F0057023C409002F8E0B401159002F6E0F5B0
:103BAF008D75C8407F281270304005C257023C40C7
:103BBF009002F6E0A3E0F58D75C8407F28127030B3
:103BCF004004C257806B9002FAE06401702EA3E0AC
:103BDF00FEA3E0F5828E83E0F58D75C8407F281235
:103BEF0070304004C2578049900300E0F58D75C8CE
:103BFF00407F281270304039C2578035E4FE900262
:103C0F00F9E0FFEEC39F50299002FBE0FCA3E0F523
:103C1F00828C83E0F58D75C8407F28127030400488
:103C2F00C257800D9002FBE475F0011223C40E8081
:103C3F00CD75C850E5C830E41B53B1F8900301E0CF
:103C4F007002A3E0600E90030174FFF5F01223C41D
:063C5F0080E280E0A257A4
:013C6500223C
:0A30A400AA079002ECECF0A3EDF097
:1030AE00D256E4900322F0A374BBF0A37480F09088
:1030BE0002F4EAF0A3EDF0EA4401A3F09002EFE08F
:1030CE00D39400500302325A43E6C043D10143C8A1
:1030DE000175C8607F08127030400C7F101270307E
:1030EE004005C2560232378A8D75C8407F1812705D
:1030FE00304005C256023237EBB401159002ECE0B7
:10310E00F58D75C8407F281270304005C2560232C8
:10311E00379002ECE0A3E0F58D75C8407F28127061
:10312E00304005C25602323775C8607F08127030C3
:10313E00400C7F101270304005C256023237EA44FE
:10314E0001F58D75C8407F401270304005C25602A1
:10315E003237E49002F3F09002EFE0FF9002F3E0DA
:10316E00FEC39F50579002F0E07031EF14B5060A7F
:10317E0075C8407F58127030800875C8447F501251
:10318E0070309002F1E0FEA3E0F5828E83E58DF0C3
:10319E009002F1E475F0011223C4801875C8447FC3
:1031AE00501270309002F3E024F7F582E43402F509
:1031BE0083E58DF09002F3E004F0809B9002F0E046
:1031CE006401706575C8407F58127030900322E517
:1031DE008DF07B017A0279F49002EFE02403FD1268
:1031EE0071C0900322E0B5073EE49002F3F0900226
:1031FE00EFE0FF9002F3E0FEC39F502D74F72EF523
:10320E0082E43402F583E0FF9002F1E0FCA3E0F5E6
:10321E00828C83EFF09002F1E475F0011223C490DA
:10322E0002F3E004F080C7C25675C850E5C830E41A
:10323E001B53B1F8900323E07002A3E0600E9003DD
:0E324E002374FFF5F01223C480E280E0A25644
:01325C00224F
:1072410075C632E4F5E6F5D1758A7043D10675C885
:07725100407589FFF58D2255
:1071DC0075C432E4F587759850759D7F759C647500
:0C71EC009E04439D80759A0A759BFF224B
:031023000262E680
:1062E600C0E0C0F0C083C082C0D075D000C000C07E
:0D62F60001C002C003C004C005C006C007FF
:10630300C086758600309807C298AF9912529430B0
:096313009905C299124EB8D0861A
:10631C00D007D006D005D004D003D002D001D000D5
:0B632C00D0D0D082D083D0F0D0E0327F
:103DAA00FFFFFFFFF07FDFCDD0DAC222B4F4A8C252
:103DBA009D769300894E804F77F770386906625670
:103DCA005C1F565650F44BF1474642EC3EDD3B141D
:103DDA003728343F312A2E462B97291226B62481BA
:103DEA002270207F1EAE1CFA1B6119E11878172673
:103DFA0015E714BC13A2129911A010B50FD80F0819
:103E0A000E440D8A0CDC0C370B9C0B090A7E09FB4D
:103E1A00097E090A089B083207CF0770071706C3ED
:103E2A000673062705DF059B055A051D04E204AB48
:103E3A0004770445041503E803BC0393036C0346A3
:103E4A000325030302E302C502A8028C0271025889
:103E5A0002400229021301FE01EA01D701C501B39A
:103E6A0001A301930183017501670159014D0140C5
:103E7A0001350129011F0114010A010100F800EFAF
:103E8A0000E600DE00D700CF00C800C100BA00B4C7
:103E9A0000AE00A800A2009D00980092008E008942
:103EAA0000840080007C007800740070006D006956
:103EBA00006600630060005D005A0057005400521B
:103ECA00004F004D004A00480046004400420040AE
:103EDA00003E003C003B0039003700360035003414
:023EEA000032A4
:031000000270ED8E
:1070ED0075819F007808760008B8A0FAE49000003A
:1070FD00F0A3A882A983B8DCF7B907F4000258768B
:102D1D00A2AF9253C2AF900234E0FFA3E09003271D
:102D2D00CFF0A3EFF090022C12259A9003451226B6
:102D3D000090023012259A900378122600900236E8
:102D4D00E0FFA3E0900366CFF0A3EFF09002201216
:102D5D00259A90037D122600900224E0FFA3E090B7
:102D6D000376CFF0A3EFF090021EE0FEA3E0FFE4A8
:102D7D00FCFD90034F122600851117851218850F43
:102D8D001585101690036112262500000000E490B1
:102D9D000374F0A3F0A25392AF90034E741EF09003
:102DAD00036D745AF0A3740BF0A3740FF0900368C5
:102DBD00122625FFFF7748E490036CF09003710411
:102DCD00F09003897414F090033E743EF0A3748068
:102DDD00F0A3E4F0A37411F09003727406F0A374E1
:102DED0022F090038B743CF0900003E02438FE90A9
:102DFD000002E034FF900325F0A3CEF09003597448
:102E0D000FF0900360740AF0900014E0FFA3E090BF
:102E1D000381CFF0A3EFF090034D745AF0E513FB4F
:102E2D007A007C117D94FF7E0012235DE4FCFD9001
:102E3D00032F1226007C0B7DB8AF037E0012235D9D
:102E4D00E4FCFD900355122600900365743CF09050
:102E5D00038A7414F0900333740FF090037C741490
:102E6D00F0900370740AF0900329122625000000DB
:102E7D0028900344741EF0900342740BF0A3744128
:102E8D00F0900353740BF0A37441F0900383E4F0BE
:102E9D00A37432F0900349E4F0A37405F090033A63
:102EAD00E4F0A37469F0900385E4F0A37464F090EA
:102EBD00034BE4F0A3741EF090033CE4F0A37462A2
:102ECD00F09003877401F0A37490F090035EE4F02A
:042EDD00A3744BF09F
:012EE10022CE
:10633700A2AF9253C2AF900327E0FFA3E0900234CD
:10634700CFF0A3EFF090034512259A90022C122666
:106357000090037812259A90023012260090036667
:10636700E0FFA3E0900236CFF0A3EFF0A251922214
:10637700A25292209000B9E024FF9221A25392AF3B
:0163870022F3
:0673F7005AA569963CC393
:10415D007F647E00E49002BBF09002BBE0FDC3944F
:10416D000A400302427BED25E02402F582E434008F
:10417D00F583E0FCA3E0D39518EC951750030242AC
:10418D00729002BBE0705790007AE0FCA3E0FDD383
:10419D009518EC95175003301906E4FEFF02427B8B
:1041AD00C3E5189DFFE5179CFE7C007D0A1226884D
:1041BD00EEC0E0EFC0E090007AE0FEA3E0FFC39018
:1041CD000003E09FFF900002E09EFECBEFCBFAE4F0
:1041DD00F9F8D0E0FFD0E0FE12248002427B90027D
:1041ED00BBE025E02400F582E43400F583E0FEA376
:1041FD00E0FFC3E5189FFFE5179EFE7C007D0A12C8
:10420D002688ECC0E0EDC0E0EEC0E0EFC0E090022B
:10421D00BBE0FF25E02400F582E43400F583E0FCEB
:10422D00A3E0FDEF25E02402F582E43400F583E000
:10423D00FEA3E0C39DFFEE9CFECBEFCBFAE4F9F8B5
:10424D00D0E0FFD0E0FED0E0FDD0E0FC122480CD28
:10425D00EFCDCCEECC9002BBE075F00AA42DFFE5BE
:0F426D00F03CFE80099002BBE004F002416622A3
:103591009002BBEEF0A3EFF09000AAE0F9FDD3EFAB
:1035A1009DEE9400500302366A90036DE0FF900295
:1035B100BBE0FCA3E0FDD39FEC94004078ED946464
:1035C100EC940050709002BBE0FAA3E0FBC374647A
:1035D1009BFFE49AFE7C007D0A12235DE9FDC3EBAB
:1035E1009DFDEA9CFCD3ED9FEC9E50030236FF90BB
:1035F10002BBE0FEA3E0FF9000AAF07C007D0A126E
:10360100235D9003AAEEF0A3EFF09002BBE0FEA3CE
:10361100E0FFE4FD90001AE0F8A3E0F9A3E0FAA3CB
:10362100E0FB1223F5E47B64FAF9F81224809000A0
:10363100AB122600229002BBE07004A3E064646038
:10364100030236FF9000AA7464F09003AA7403F099
:10365100A374E8F090001AE0FCA3E0FDA3E0FEA350
:10366100E0FF9000AB122600229000AAE0FD90023C
:10367100BBE0FEA3E0FFC3ED9FFDE49EFC90034E83
:10368100E0FBD3ED9BEC9400403F9000AAEFF07C6F
:10369100007D0A12235D9003AAEEF0A3EFF09002E1
:1036A100BBE0FEA3E0FFE4FD90001AE0F8A3E0F91F
:1036B100A3E0FAA3E0FB1223F5E47B64FAF9F81224
:1036C10024809000AB122600229002BBE07002A37E
:1036D100E0702B9000AA04F09003AAE4F0A3740A0E
:1036E100F0E47B64FAF9F890001AE0FCA3E0FDA392
:0F36F100E0FEA3E0FF1224809000AB122600221F
:10370000122D1D12415D9002B9EEF0A3EFF0E47F9F
:10371000E87E03FDFC9000ABE0F8A3E0F9A3E0FA3B
:10372000A3E0FB1223F590001AE0F8A3E0F9A3E070
:10373000FAA3E0FB1224809003AAEEF0A3EFF0902E
:1037400002B9E0FEA3E0FF1235919000AAE0FF7EEF
:1037500000900327EEF0FAA3EFF0FB90001AE0FCD4
:10376000A3E0FDA3E0FEA3E0FF900345122600CFF7
:10377000EBCF7E00E4FCFD900345E0F8A3E0F9A365
:10378000E0FAA3E0FB1223F5E47B64FAF9F81224D3
:10379000809003781226009000ABE0FCA3E0FDA32C
:1037A000E0FEA3E0FF90035A122600900336122693
:1037B00025000000009003A8E0FFA3E090032DCFB8
:1037C000F0A3EFF0E47830F608F67838F608F678EB
:1037D0003412260C000000009003AE1226250000D3
:1037E0000000E490039EF0A3F09003B4F0A3F090E7
:1037F00003ACF0A3F0C252C24EC2509003A7F090A7
:1038000003A6F0783AF608F67832F608F69003AA9E
:10381000E0FFA3E09003B2CFF0A3EFF0C251C24D9E
:103820009003B612262500000000E49003A8F0A340
:10383000F0900390122625000000009003991226B4
:10384000250000000090039412262500000000E4EB
:1038500090039DF0900398F0C24F90038C122625A0
:08386000000000001263372292
:10445A0012415D9002B9EEF0A3EFF0900333E0FF52
:10446A00E4FCFDFE90001AE0F8A3E0F9A3E0FAA349
:10447A00E0FB1223F5E47B0AFAF9F8122480C8EC6F
:10448A00C8C9EDC9CAEECACBEFCB90037DE0FCA345
:10449A00E0FDA3E0FEA3E0FFD3122543500302454B
:1044AA003090037CE0FF7E009002B9E0FCA3E0FDBF
:1044BA00D39FEC9E4070D3900382E09518900381BD
:1044CA00E095174061ED9FFBEC9EFA9003AAE0FE8F
:1044DA00A3E0FF7C007D0A12236FC3EF9BEE9A5084
:1044EA0045900370E0FFC39002BAE09FFF9002B9C3
:1044FA00E09400FE7C007D0A12235D9003AAEEF090
:10450A00A3EFF0E4FD90001AE0F8A3E0F9A3E0FAC3
:10451A00A3E0FB1223F5E47BE87A03F9F81224807E
:07452A009000AB12260022F5
:101C7A00122D1D900342E0FEA3E0FFD3900377E00C
:101C8A009F900376E09E401EE4FFFEFDFC900399C0
:101C9A00E0F8A3E0F9A3E0FAA3E0FBD312252D4074
:101CAA0005301802D252C3900382E095189003813E
:101CBA00E095175012900398E004F0E09405400E66
:101CCA007405F0D24E8007C24EE4900398F090005B
:101CDA0028E0FEA3E0FFEE3395E0FDFC90037DE0F3
:101CEA00F8A3E0F9A3E0FAA3E0FBD312252D5003F1
:101CFA00021EE2E49003B4F0A3F09003ACF0A3F068
:101D0A0090039DE004F0E0D3940540057405F0D2F9
:101D1A004F9000B9E06010D251E4F09003B6122659
:101D2A002500000000C24D900374E0FEA3E0FFEE20
:101D3A003395E0FDFC900281E0F8A3E0F9A3E0FA14
:101D4A00A3E02FFFEA3EFEE93DFDE83CFC9003904C
:101D5A00122600E4FFFEFDFC900390E0F8A3E0F9F0
:101D6A00A3E0FAA3E0FBD312252D4021900281E0E3
:101D7A00A3E0A3E0FEA3E0FF900375E02FFF90032A
:101D8A0074E03EFE783BEF26F618EE36F6C3783B53
:101D9A00E6941018E6940E5003021E2C0874F026DE
:101DAA00F61874F136F690001AE0FCA3E0FDA3E001
:101DBA00FEA3E0FF9000ABE0F8A3E0F9A3E0FAA3EA
:101DCA00E0FBC312254350219000ABE0FCA3E0FDE9
:101DDA00A3E0FEA3E02401FFE43EFEE43DFDE43C73
:101DEA00FC9000AB122600801490001AE0FCA3E0DD
:101DFA00FDA3E0FEA3E0FF9000AB12260030518D58
:101E0A009003B6E0FCA3E0FDA3E0FEA3E02401FFFB
:101E1A00E43EFEE43DFDE43CFC9003B612260002DB
:101E2A001D97900342E0FEA3E0FFD3900377E09F63
:101E3A00900376E09E404490006AE0FEA3E0FFEE45
:101E4A003395E0FDFC900281E0F8A3E0F9A3E0FA03
:101E5A00A3E0FBC312252D5022C3900069E0951818
:101E6A00900068E09517501390006CE0FF9003A76C
:101E7A00E004F0C39F4004EFF0D25290006AE0FE03
:101E8A00A3E0FFEE3395E0FDFC900281E0F8A3E0C9
:101E9A00F9A3E0FAA3E0FBC312252D503590034FB6
:101EAA00E0FCA3E0FDA3E0FEA3E0FF90032FE0F82F
:101EBA00A3E0F9A3E0FAA3E0FBC312254350139071
:101ECA000365E0FF9003A6E004F0C39F4004EFF02F
:101EDA00D25012445A022220900028E0FEA3E0FFCA
:101EEA00C3E49FFFE49EFE3395E0FDFC90037DE092
:101EFA00F8A3E0F9A3E0FAA3E0FBC312252D4003FF
:101F0A000220D7E49003A7F09003A6F0C250C25271
:101F1A009003ACF0A3F09003B5F090039DF0C24F8C
:101F2A00900361E0FCA3E0FDA3E0FEA3E0FF9002C2
:101F3A0081E0F8A3E0F9A3E0FAA3E02FFBEA3EFA76
:101F4A00E93DF9E83CF8900374E0FEA3E0FFEE33C4
:101F5A0095E0FDFCEB2FFFEA3EFEE93DFDE83CFC87
:101F6A00900390122600900390E0FCA3E0FDA3E00A
:101F7A00FEA3E0FFEC33500AC37833E69FF618E677
:101F8A009EF6C37833E6941018E6940E50030220A6
:101F9A006CC37833E6941018E6940E40670874F020
:101FAA0026F61874F136F69000B3E0FCA3E0FDA320
:101FBA00E0FEA3E02401FFE43EFEE43DFDE43CFC38
:101FCA009000B3122600E47F01FEFDFC9000ABE016
:101FDA00F8A3E0F9A3E0FAA3E0FBD312254340B14A
:101FEA009000ABE0FCA3E0FDA3E0FEA3E024FFFF2A
:101FFA00EE34FFFEED34FFFDEC34FFFC9000AB1233
:10200A002600808D90001EE0FCA3E0FDA3E0FEA365
:10201A00E0FF9000B3E0F8A3E0F9A3E0FAA3E0FB45
:10202A00C3122543403C9000B3E0FCA3E0FDA3E0CB
:10203A00FEA3E0FF90001EE0F8A3E0F9A3E0FAA3F4
:10204A00E0FBEF9BFFEE9AFEED99FDEC98FC900009
:10205A00B3122600900023E004F07006900022E0FC
:10206A0004F0900353E0FEA3E0FFD3900377E09FD0
:10207A00900376E09E50030222209000AFE0FCA37A
:10208A00E0FDA3E0FEA3E0FF900281E0F8A3E0F9FF
:10209A00A3E0FAA3E0FBD312252D5003022220D39A
:1020AA0090007BE0951690007AE095155003022285
:1020BA002090007CE0FF9003B4E004F09F500302FC
:1020CA002220EFF09000B97401F0022220900374EC
:1020DA00E0FAA3E0FBFFCEEACEEE3395E0FDFC3357
:1020EA0040030221CAC37833E69BFF18E69AFEF63C
:1020FA0008EFF6C39410EE940E50030221CA74F04E
:10210A0026F61874F136F69000B3E0FCA3E0FDA3BE
:10211A00E0FEA3E02401FFE43EFEE43DFDE43CFCD6
:10212A009000B3122600E47F01FEFDFC9000ABE0B4
:10213A00F8A3E0F9A3E0FAA3E0FBD3122543402277
:10214A009000ABE0FCA3E0FDA3E0FEA3E024FFFFC8
:10215A00EE34FFFEED34FFFDEC34FFFC9000AB12D1
:10216A00260090001EE0FCA3E0FDA3E0FEA3E0FF32
:10217A009000B3E0F8A3E0F9A3E0FAA3E0FBC312EE
:10218A002543403C9000B3E0FCA3E0FDA3E0FEA39E
:10219A00E0FF90001EE0F8A3E0F9A3E0FAA3E0FB59
:1021AA00EF9BFFEE9AFEED99FDEC98FC9000B312BE
:1021BA002600900023E004F07006900022E004F06C
:1021CA0090038BE0FF9003ACE475F0011223C4FC8A
:1021DA00C3E5F09FEC9400403A900353E0FEA3E07D
:1021EA00FFD3900377E09F900376E09E4025D3903B
:1021FA00007BE0951690007AE09515401690007CD9
:10220A00E0FF9003B5E004F09F4008EFF09000B9BA
:10221A007401F01226B5E47FE87E03FDFC9000AB62
:10222A00E0F8A3E0F9A3E0FAA3E0FB1223F590009B
:10223A001AE0F8A3E0F9A3E0FAA3E0FB12248090E5
:10224A0003AAEEF0A3EFF0900028E0FEA3E0FFC39C
:10225A00E49FFFE49EFE3395E0FDFC90037DE0F8E9
:10226A00A3E0F9A3E0FAA3E0FBC312252D400C205A
:10227A001509201A06201B03301C02C251121056DF
:10228A009000AAE0FF7E00900327EEF0FAA3EFF099
:10229A00FB90001AE0FCA3E0FDA3E0FEA3E0FF90A0
:1022AA000345122600CFEBCF7E00E4FCFD900345E8
:1022BA00E0F8A3E0F9A3E0FAA3E0FB1223F5E47B3C
:1022CA0064FAF9F81224809003781226009000220A
:1022DA00E0FFA3E0900366CFF0A3EFF09003AAE03B
:1022EA00FFA3E09003B2CFF0A3EFF0900390E0FCDD
:1022FA00A3E0FDA3E0FEA3E0FF900399122600905D
:10230A0000ABE0FCA3E0FDA3E0FEA3E0FF90035ACC
:10231A001226009003AEE0FCA3E0FDA3E0FEA3E0DA
:10232A00FF9003361226009003A8E0FFA3E0900373
:0A233A002DCFF0A3EFF0126337225D
:106E8F00122D1D90038C1225BF900329E0F8A3E06B
:106E9F00F9A3E0FAA3E0FBC3122543501490032992
:106EAF00E0FCA3E0FDA3E0FEA3E0FF90038C12261D
:056EBF00001263372200
:10290D009005F5E4F0A37464F0122D1D12415D9055
:10291D0005F5EEF0A3EFF04E702E9000AA04F090A6
:10292D0003AAE4F0A3740AF0E47B64FAF9F89000CA
:10293D001AE0FCA3E0FDA3E0FEA3E0FF12248090CB
:10294D0000AB122600022A17900329E0FCA3E0FD3C
:10295D00A3E0FEA3E0FF90038CE0F8A3E0F9A3E071
:10296D00FAA3E0FBC3122543400E9005F5E0FEA34C
:10297D00E0FF123591022A17E47F64FEFDFC900002
:10298D001AE0F8A3E0F9A3E0FAA3E0FB1223F59017
:10299D0000ABE0F8A3E0F9A3E0FAA3E0FB1224807A
:1029AD00C8ECC8C9EDC9CAEECACBEFCB90034EE057
:1029BD00FF9005F6E02FFF9005F5E03400FEE4FCF6
:1029CD00FDD312254340439005F5E0FAA3E0FB7CCF
:1029DD00007D0AFFCEEACE12235D9003AAEEF0A38E
:1029ED00EFF0CFEBCFCEEACEE4FD90001AE0F8A3E6
:1029FD00E0F9A3E0FAA3E0FB1223F5E47B64FAF916
:102A0D00F81224809000AB122600E47830F608F618
:102A1D007838F608F6783412260C00000000900382
:102A2D00AE12262500000000E490039EF0A3F09066
:102A3D0003B4F0A3F09003ACF0A3F0C252C24EC2A7
:102A4D00509003A7F09003A6F0783AF608F6783286
:102A5D00F608F69003AAE0FFA3E09003B2CFF0A32F
:102A6D00EFF0C251C24D9003B612262500000000B2
:102A7D00E49003A8F0A3F090039012262500000027
:102A8D000090039912262500000000900394122651
:102A9D002500000000E490039DF0900398F0C24FD4
:102AAD0090038C122625000000009000AAE0FF7E06
:102ABD0000900327EEF0FAA3EFF0FB90001AE0FC74
:102ACD00A3E0FDA3E0FEA3E0FF900345122600CF97
:102ADD00EBCF7E00E4FCFD900345E0F8A3E0F9A305
:102AED00E0FAA3E0FB1223F5E47B64FAF9F8122473
:102AFD00809003781226009000ABE0FCA3E0FDA3CC
:102B0D00E0FEA3E0FF90035A122600900336122632
:102B1D002500000000E490032DF0A3F0126337228E
:1026B500305109305206C251D24D802130521E9000
:1026C50003AA7403F0A374E8F090001AE0FCA3E0F9
:1026D500FDA3E0FEA3E0FF9000AB122600304D0302
:1026E5000227659000B7E0FCA3E0FD900022E0FE24
:1026F500A3E0FFC39DFDEE9CFCC390035FE09D90AE
:10270500035EE09C400302290C20520302290C12AF
:102715005F77E4FCFDFE90001AE0F8A3E0F9A3E082
:10272500FAA3E0FB1223F5ECC0E0EDC0E0EEC0E05B
:10273500EFC0E09000B7E0FEA3E0FF125F77CBEFBC
:10274500CBE4FAF9F8D0E0FFD0E0FED0E0FDD0E030
:10275500FC1224809003B61226000228C10228C16B
:10276500C24DE47F32FEFDFC900016E0F8A3E0F9CF
:10277500A3E0FAA3E0FB1223F5E47B64FAF9F8126F
:1027850024809002B91226009002B9E0FCA3E0FD76
:10279500A3E0FEA3E0FF9003B6E0F8A3E0F9A3E011
:1027A500FAA3E02FFFEA3EFEE93DFDE83CFC900080
:1027B50016E0F8A3E0F9A3E0FAA3E0FBC312254372
:1027C500400302290C900344E0FFE4FCFDFE900069
:1027D5001AE0F8A3E0F9A3E0FAA3E0FB1223F5E47D
:1027E5007B64FAF9F81224809002B912260090024F
:1027F500B9E0FCA3E0FDA3E0FEA3E0FF90001AE032
:10280500F8A3E0F9A3E0FAA3E02FFFEA3EFEE93DD5
:10281500FDE83CFC9003B6E0F8A3E0F9A3E0FAA3D9
:10282500E0FBD3122543402E9002B9E0FCA3E0FD66
:10283500A3E0FEA3E0FF90001AE0F8A3E0F9A3E00F
:10284500FAA3E02FFFEA3EFEE93DFDE83CFC9003DC
:10285500B612260080669002B9E0FCA3E0FDA3E075
:10286500FEA3E0FF9003B6E0F8A3E0F9A3E0FAA326
:10287500E02FFFEA3EFEE93DFDE83CFC90001AE052
:10288500F8A3E0F9A3E0FAA3E0FBD3122543402C1B
:102895009002B9E0F8A3E0F9A3E0FAA3E0FB900009
:1028A5001AE0FCA3E0FDA3E0FEA3E09BFFEE9AFE89
:1028B500ED99FDEC98FC9003B61226009003B6E066
:1028C500FCA3E0FDA3E0FEA3E0FF90001A122600A2
:1028D5009003AA7403F0A374E8F090001AE0FCA337
:1028E500E0FDA3E0FEA3E0FF9000AB122600900000
:1028F50022E0FFA3E09000B7CFF0A3EFF09003B67E
:0829050012262500000000224B
:105F7700C3900388E09F900387E09E500479558083
:105F870048C3900386E09F900385E09E50169003D8
:105F97004BE0FCA3E0FD12236F90033CE0A3E0C3BA
:105FA7009FF98025C3900384E09F900383E09E5070
:105FB70016900349E0FCA3E0FD12236F90033AE03B
:0D5FC700A3E0C39FF980027964CFE9CF22E7
:10105600E49002B9F0A3F0FFA3F0A3F0A3F090038D
:10106600A0E0645A6028A2AF9253C2AF75A701E40C
:10107600EF90124093FE74A02FF582E43403F583BB
:10108600EEF00FEFB406E9E4F5A7A25392AF900392
:10109600A5E064C36003021C48FF74A02FF582E438
:1010A6003403F583E0FEEF9073F7936E6003021C42
:1010B600480FEFB406E48003021C48900028E0FEC7
:1010C600A3E0FFEE3395E0FDFC90037DE0F8A3E09E
:1010D600F9A3E0FAA3E0FBD312252D50030214F185
:1010E600204F030214F1E47830F608F67838F60853
:1010F600F69000AAE0D394634003021C48C3900311
:1011060082E09518900381E09517401E90034DE00C
:10111600FF7E007C007D0A12235DD39003ABE09F27
:101126009003AAE09E50030213C9304E5A90034D15
:10113600E0FBFF7E007C007D0A12235D9003ABE09E
:101146002496FD9003AAE03400FCC3ED9FEC9E506C
:1011560036EBFF7E007C007D0A12235DEEF0A3EFE6
:10116600F0CFEBCFE4FDFE90001AE0F8A3E0F9A380
:10117600E0FAA3E0FB1223F5E47B64FAF9F8122403
:10118600809000AB12260090034FE0FCA3E0FDA385
:10119600E0FEA3E0FF90032FE0F8A3E0F9A3E0FA56
:1011A600A3E0FBD3122543500302123090034FE015
:1011B600F8A3E0F9A3E0FAA3E0FB90032FE0FCA379
:1011C600E0FDA3E0FEA3E09BFBEE9AFAED99F9ECB5
:1011D60098F8900389E0FFE4FCFDFE1223F5E47B1A
:1011E6000AFAF9F81223F5EEC0E0EFC0E090001419
:1011F600E0FEA3E0FFC3900069E09FFF900068E077
:101206009EFECBEFCBFAE4F9F8D0E0FFD0E0FE1279
:101216002480EFC0E0AF13CBEFCBE4FAF9F8D0E0CF
:10122600FF122480900394122600C3900063E09579
:1012360018FF900062E09517FE900389E0FD7C00A0
:10124600122688E47B0AFAF9F81223F5EEC0E0EFDD
:10125600C0E0900014E0FEA3E0FFC3900069E09FA9
:10126600FF900068E09EFECBEFCBFAE4F9F8D0E001
:10127600FFD0E0FE1224809002BE12260090039456
:10128600E0FCA3E0FDA3E0FEA3E0FF9002BEE0F8D1
:10129600A3E0F9A3E0FAA3E0FBC3122543501490A0
:1012A60002BEE0FCA3E0FDA3E0FEA3E0FF900394F2
:1012B600122600E47F24FEFDFC90001AE0F8A3E06D
:1012C600F9A3E0FAA3E0FB1223F5900394E0F8A358
:1012D600E0F9A3E0FAA3E0FB1223F5EEC0E0EFC0CD
:1012E600E09000AAE0FFC374659FFFE49400FECB84
:1012F600EFCBFAE4F9F8D0E0FFD0E0FE122480E468
:101306007B0AFAF9F81224809003941226009000C2
:101316006AE0FEA3E0FFEE3395E0FDFC900390E06B
:10132600F8A3E0F9A3E0FAA3E0FBD312252D406C65
:10133600900390E0FCA3E0FDA3E0FEA3E0FFC8EC71
:10134600C8A3E0FCA3E0FDA3E0FEA3E0FF12248017
:10135600ECC0E0EDC0E0EEC0E0EFC0E090006AE077
:10136600FEA3E0FFFBCAEECAEA3395E0F9F8900364
:1013760090E0FCA3E0FDA3E0FEA3E0C39BFFEE9A92
:10138600FEED99FDEC98FCD0E0FBD0E0FAD0E0F958
:10139600D0E0F81223F5900394122600900063E043
:1013A60024FFFF900062E034FFFEC3E5189FE517B7
:1013B6009E50030214839003941226250000000019
:1013C6000214839003AAE0FEA3E0FF7C007D0A12CC
:1013D600236FEF2401FFE43EFE9000AAE0FB7A00B3
:1013E600C39FEA9E503C9003AAE0FEA3E0FF7C0068
:1013F6007D0A12236FEB2401FDEA33FCD3ED9FEC4B
:101406009E401FE47F24FEFDFC90001AE0F8A3E056
:10141600F9A3E0FAA3E0FB1223F590039412260049
:10142600805B9000ABE0F8A3E0F9A3E0FAA3E0FB51
:1014360090001AE0FCA3E0FDA3E0FEA3E0C39BFF3F
:10144600EE9AFEED99FDEC98FCE47B107A0EF9F825
:101456001223F5EEC0E0EFC0E09000AAE0FFC374EF
:10146600649FFFE49400FECBEFCBFAE4F9F8D0E0FA
:10147600FFD0E0FE12248090039412260090039081
:10148600E0FCA3E0FDA3E0FEA3E0FFFBCAEECAC9B1
:10149600EDC9C8ECC8A3E0FCA3E0FDA3E0FEA3E011
:1014A600FF1224809002BCEEF0A3EFF02050033030
:1014B600520D90038AE0FF9002BCE4F0A3EFF09097
:1014C60003A8E475F0011223C4FEC39002BDE095A3
:1014D600F09002BCE09E4003021C489000AAE00483
:1014E600F0E49003A8F0A3F0021C48900028E0FE68
:1014F600A3E0FFC3E49FFFE49EFE3395E0FDFC906E
:10150600037DE0F8A3E0F9A3E0FAA3E0FBC312250C
:101516002D4003021BE89000AAE094015003021C30
:1015260048900325E0FEA3E0FFAD137C0012268859
:1015360090034FE0F8A3E0F9A3E0FAA3E0FBC3129F
:101546002543402DD390007BE0951690007AE095D8
:1015560015501E900359E0FF7E007C007D0A122381
:101566005DC39003ABE09F9003AAE09E4003021880
:101576000B90036EE0FEA3E0FFD3900377E09F900D
:101586000376E09E500302180B900368E0FCA3E08C
:10159600FDA3E0FEA3E0FF90037DE0F8A3E0F9A33E
:1015A600E0FAA3E0FBD312252D500302180B78397D
:1015B600E61846700302180B900399E0FCA3E0FDC1
:1015C600A3E0FEA3E024D0FFEE3407FEE43DFDE4F5
:1015D6003CFC900390E0F8A3E0F9A3E0FAA3E0FB5B
:1015E600C312252D400302180B900399E0FCA3E0DB
:1015F600FDA3E0FEA3E02430FFEE34F8FEED34FF59
:10160600FDEC34FFFC900390E0F8A3E0A3E0A3E038
:10161600D312252D500302180B900360E07E00259F
:1016260016FFEE3515FEC3EF783996EE1896400391
:101636000217FA90039EE0FEA3E0FF9400EE9400EA
:1016460050030217FAEF9401EE9400500890039E9F
:10165600E4F0A304F090034FE0FCA3E0FDA3E0FE5A
:10166600A3E0FF78341225A6D312254350030217B0
:1016760013900355E0F8A3E0F9A3E0FAA3E0FB908A
:10168600034FE0FCA3E0FDA3E0FEA3E09BFBEE9A84
:10169600FAED99F9EC98F890039EE0FEA3E0FFE4DA
:1016A600FCFD1223F5ECC0E0EDC0E0EEC0E0EFC0BB
:1016B600E090034FE0F8A3E0F9A3E0FAA3E0FBE82B
:1016C600C0E0783412258ED0E0F8C3EF9BFBEE9A8B
:1016D600FAED99F9EC98F8D0E0FFD0E0FED0E0FD05
:1016E600D0E0FC122480EEC0E0EFC0E09000AAE05B
:1016F60024FFFFE434FFFECBEFCBFAE4F9F8D0E0A9
:10170600FFD0E0FE1224809003941226009000740D
:10171600E0FEA3E0FFC3E5169FFFE5159EFE9003DE
:101726009EE0FCA3E0FD122688EEC0E0EFC0E0C319
:101736007839E69516FF18E69515FECBEFCBFAE459
:10174600F9F8D0E0FFD0E0FE122480EEC0E0EFC052
:10175600E09000AAE024FFFFE434FFFECBEFCBFAD3
:10176600E4F9F8D0E0FFD0E0FE1224809002BE1229
:101776002600900394E0FCA3E0FDA3E0FEA3E0FFB7
:101786009002BEE0F8A3E0F9A3E0FAA3E0FBC312DF
:10179600254350149002BEE0FCA3E0FDA3E0FEA3A7
:1017A600E0FF9003941226007838A61508A6169036
:1017B600034FE0FCA3E0FDA3E0FEA3E0FF783412B4
:1017C60025F4E490039EF0A3F0900394E0F8A3E0E0
:1017D600F9A3E0FAA3E0FB900390E0FCA3E0FDA3ED
:1017E600E0FEA3E0FF12251F1223F59003941226B4
:1017F60000021B7690039FE004F0700690039EE0C3
:1018060004F0021B767838A61508A61690034FE05A
:10181600FCA3E0FDA3E0FEA3E0FF78341225F4E488
:1018260090039EF0A3F090036EE0FEA3E0FFC3904A
:101836000377E09F900376E09E4021900368E0FCEA
:10184600A3E0FDA3E0FEA3E0FF90037DE0F8A3E0A4
:10185600F9A3E0FAA3E0FB12252D501D90001AE033
:10186600FCA3E0FDA3E0FEA3E0FF9003AE1226007A
:10187600E47830F608F60219FA7830E6FE08E6FF54
:101886002414FDE43EFC900376E0FAA3E0FBD39D2E
:10189600EA9C5011EB2414FDE43AFCD3EF9DEE9C38
:1018A60050030219FA900376E0FEA3E0FF7830EECB
:1018B600F608EFF62487FFEE34F59002B9F0A3EFB1
:1018C600F0900340E0FEA3E0FFFBCAEECAE4F9F89D
:1018D6009002B9E0FEA3E0FFEE3395E0FDFC122393
:1018E600F5C8ECC8C9EDC9CAEECACBEFCB90033E2A
:1018F600E0FEA3E0FFE4C3EF9BFBEE9AFAE499F95E
:10190600E498F89002B9E0FEA3E0FFEE3395E0FD1F
:10191600FC1223F5E47B107A27F9F8126AC1C8ECA9
:10192600C8C9EDC9CAEECACBEFCB900372E0FEA3DD
:10193600E0FFE4FCFDEB2FFFEA3EFEED39FDEC385F
:10194600FC90001AE0F8A3E0F9A3E0FAA3E0FB128A
:1019560023F5E47BD07A07F9F81224809003AE12BF
:10196600260090001AE0FCA3E0FDA3E0FEA3E0FF42
:101976009003AEE0F8A3E0F9A3E0FAA3E0FBD312EC
:101986002543401690001AE0FCA3E0FDA3E0FEA369
:10199600E0FF9003AE122600805AE47F06FEFDFCAF
:1019A60090001AE0F8A3E0F9A3E0FAA3E0FB122303
:1019B600F5E47B0AFAF9F81224809003AEE0F8A366
:1019C600E0F9A3E0FAA3E0FBC31225435026E47F27
:1019D60006FEFDFC90001AE0F8A3E0F9A3E0FAA3E6
:1019E600E0FB1223F5E47B0AFAF9F812248090034F
:1019F600AE1226009003AEE0F8A3E0F9A3E0FAA346
:101A0600E0FB90001AE0FCA3E0FDA3E0FEA3E0C328
:101A16009BFFEE9AFEED99FDEC98FCE47B0DFAF93E
:101A2600F81223F5E47B0AFAF9F81224809000AB49
:101A3600E0F8A3E0F9A3E0FAA3E0FBC312254350C4
:101A460020E47F24FEFDFC90001AE0F8A3E0F9A351
:101A5600E0FAA3E0FB1223F5900394122600021B82
:101A6600769000ABE0FCA3E0FDA3E0FEA3E0FF90D0
:101A760003AEE0F8A3E0F9A3E0FAA3E02FFFEA3E05
:101A8600FEE93DFDE83CFC90001AE0F8A3E0F9A36E
:101A9600E0FAA3E0FBC3EF9BFFEE9AFEED99FDECA7
:101AA60098FCE47B64FAF9F81223F59003AEE0F8AB
:101AB600A3E0F9A3E0FAA3E0FB1224809002BBEFB7
:101AC600F02401FFE433FE9000AAE0FDC39FEE641C
:101AD60080F87480985035ED2401FFE433FE9002BF
:101AE600BBE0FDD3EF9D7480F86E98401FE47F2421
:101AF600FEFDFC9003AEE0F8A3E0F9A3E0FAA3E054
:101B0600FB1223F590039412260080649000ABE04C
:101B1600FCA3E0FDA3E0FEA3E0FF9003AEE0F8A384
:101B2600E0F9A3E0FAA3E02FFFEA3EFEE93DFDE877
:101B36003CFC90001AE0F8A3E0F9A3E0FAA3E0FB6E
:101B4600C3EF9BFFEE9AFEED99FDEC98FCE47B104B
:101B56007A0EF9F81223F5EFC0E09000AAE0FFFB39
:101B6600E4FAF9F8D0E0FF122480900394122600DC
:101B7600900390E0FCA3E0FDA3E0FEA3E0FF1225A6
:101B86001FCBEFCBCAEECAC9EDC9C8ECC8A3E0FCAF
:101B9600A3E0FDA3E0FEA3E0FF1224809002BCEECA
:101BA600F0A3EFF09003A8E475F0011223C4FCD370
:101BB600E5F09FEC9E400D9000AAE014F0E490033F
:101BC600A8F0A3F030197B900371E0FF9000AAE023
:101BD600D39F506E90036CE060689000AA7401F089
:101BE6008060E47838F608F6783412260C00000097
:101BF60000E47830F608F69000AAE0D3940140425B
:101C0600900374E0FEA3E0FFEE3395E0FDFC335055
:101C1600319003AAE0FEA3E0FF7C007D0A12236F49
:101C2600CAEECACBEFCB9003B2E0FEA3E0FF7C0086
:101C36007D0A12236FD3EF9BEE9A40069000AAE02E
:101C460014F0E4FFFEFDFC900399E0F8A3E0F9A38D
:101C5600E0FAA3E0FBD312252D40093018069000C8
:101C6600AA7464F09002BCE0FFA3E0900334CFF0C6
:041C7600A3EFF022C6
:1071A300304C19204306204403304510C24CC243DF
:0D71B300C244C245C2AF12731C1200A622D6
:10F8000033270C800D480DDE0E740ED80F3C0FA070
:10F8100010041036106800000FA000000FA00000B8
:10F820000BB800000B410000006414010064055A8D
:10F83000021501300073696E6F7765616C74680042
:10F840000020231222000053483339463030340060
:10F850000000004C494F4E00000000000000000076
:10F86000005A109A10360202104000640500000B86
:10F87000B802025A0A8C0BB802020B5405FFFFB102
:10F88000E002FFFF63C002045A0FA01E465A0C9FFD
:10F890000C6D0AAB0ADD03035A0D670CD10A470A47
:10F8A000795A105400140064025A6400000BB8FF27
:10F8B000FFEC78000000000000005A7411305A0A72
:10F8C00022FFAE000100000000005A00000000000E
:10F8D0000000000000000000000000000000000028
:10F8E0000000000000000000000000000000000018
:10F8F0000000000000000000000000000000000008
:10F9000000000000000000000000000000000000F7
:10F9100000000000000000000000000000000000E7
:10F9200000000000000000000000000000000000D7
:10F9300000000000000000000000000000000000C7
:10F9400000000000000000000000000000000000B7
:10F9500000000000000000000000000000000000A7
:10F960000000000000000000000000000000000097
:10F970000000000000000000000000000000000087
:10F980000000000000000000000000000000000077
:10F990000000000000000000000000000000000067
:10F9A0000000000000000000000000000000000057
:10F9B0000000000000000000000000000000000047
:10F9C0000000000000000000000000000000000037
:10F9D0000000000000000000000000000000000027
:10F9E0000000000000000000000000000000000017
:10F9F00000000000000000000000000000005AA508
:10FA000033270C800D480DDE0E740ED80F3C0FA06E
:10FA100010041036106800000FA000000FA00000B6
:10FA20000BB800000B410000006414010064055A8B
:10FA3000021501300073696E6F7765616C74680040
:10FA4000002023122200005348333946303034005E
:10FA50000000004C494F4E00000000000000000074
:10FA6000005A109A10360202104000640500000B84
:10FA7000B802025A0A8C0BB802020B5405FFFFB100
:10FA8000E002FFFF63C002045A0FA01E465A0C9FFB
:10FA90000C6D0AAB0ADD03035A0D670CD10A470A45
:10FAA000795A105400140064025A6400000BB8FF25
:10FAB000FFEC78000000000000005A7411305A0A70
:10FAC00022FFAE000100000000005A00000000000C
:10FAD0000000000000000000000000000000000026
:10FAE0000000000000000000000000000000000016
:10FAF0000000000000000000000000000000000006
:10FB000000000000000000000000000000000000F5
:10FB100000000000000000000000000000000000E5
:10FB200000000000000000000000000000000000D5
:10FB300000000000000000000000000000000000C5
:10FB400000000000000000000000000000000000B5
:10FB500000000000000000000000000000000000A5
:10FB60000000000000000000000000000000000095
:10FB70000000000000000000000000000000000085
:10FB80000000000000000000000000000000000075
:10FB90000000000000000000000000000000000065
:10FBA0000000000000000000000000000000000055
:10FBB0000000000000000000000000000000000045
:10FBC0000000000000000000000000000000000035
:10FBD0000000000000000000000000000000000025
:10FBE0000000000000000000000000000000000015
:10FBF00000000000000000000000000000005AA506
:10234400BB010689828A83E0225002E722BBFE0297
:09235400E32289828A83E49322CA
:10235D00EF8DF0A4A8F0CF8CF0A428CE8DF0A42E94
:02236D00FE224E
:10236F00BC000BBE0029EF8DF084FFADF022E4CC52
:10237F00F875F008EF2FFFEE33FEEC33FCEE9DEC1B
:10238F00984005FCEE9DFE0FD5F0E9E4CEFD22ED61
:10239F00F8F5F0EE8420D21CFEADF075F008EF2FAB
:1023AF00FFED33FD4007985006D5F0F222C398FD9C
:0523BF000FD5F0EA2239
:1023C400C5F0F8A3E028F0C5F0F8E58215827002A4
:0623D4001583E038F02241
:0D23DA00EF2BFFEE3AFEED39FDEC38FC2252
:0E23E700C3EF9BFFEE9AFEED99FDEC98FC22F1
:1023F500E88FF0A4CC8BF0A42CFCE98EF0A42CFC87
:102405008AF0EDA42CFCEA8EF0A4CDA8F08BF0A404
:102415002DCC3825F0FDE98FF0A42CCD35F0FCEB63
:102425008EF0A4FEA9F0EB8FF0A4CFC5F02ECD3928
:0F243500FEE43CFCEAA42DCE35F0FDE43CFC2295
:1024440075F008758200EF2FFFEE33FECD33CDCC4F
:1024540033CCC58233C5829BED9AEC99E5829840D2
:102464000CF582EE9BFEED9AFDEC99FC0FD5F0D6AF
:10247400E4CEFBE4CDFAE4CCF9A88222B800C1B9D9
:102484000059BA002DEC8BF084CFCECDFCE5F0CB17
:10249400F97818EF2FFFEE33FEED33FDEC33FCEB50
:1024A40033FB10D703994004EB99FB0FD8E5E4F90B
:1024B400FA227818EF2FFFEE33FEED33FDEC33FCF8
:1024C400C933C910D7059BE99A4007EC9BFCE99AEC
:1024D400F90FD8E0E4C9FAE4CCFB2275F010EF2F31
:1024E400FFEE33FEED33FDCC33CCC833C810D70731
:1024F4009BEC9AE899400AED9BFDEC9AFCE899F86C
:0E2504000FD5F0DAE4CDFBE4CCFAE4C8F922FE
:106AC100C2D5E830E70FB2D5E4C39BFBE49AFAE400
:106AD10099F9E498F8EC30E717B2D5126AF7122465
:106AE10080E4C39BFBE49AFAE499F9E498F8800303
:106AF10012248030D50DE4C39FFFE49EFEE49DFD8A
:046B0100E49CFC22F2
:0D251200EF4BFFEE4AFEED49FDEC48FC22C8
:0E251F00C3E49FFFE49EFEE49DFDE49CFC22CD
:10252D00EB9FF5F0EA9E42F0E99D42F0EC6480C825
:06253D0064809845F022C5
:10254300EB9FF5F0EA9E42F0E99D42F0E89C45F0EE
:012553002265
:10255400E8600FECC313FCED13FDEE13FEEF13FF65
:03256400D8F12289
:10256700E86010ECA2E713FCED13FDEE13FEEF138A
:04257700FFD8F02277
:10257B00E8600FEFC333FFEE33FEED33FDEC33FCBE
:03258B00D8F12262
:0C258E00E6FC08E6FD08E6FE08E6FF2279
:0C259A00E0FCA3E0FDA3E0FEA3E0FF22B4
:0D25A600E6FB08E6F908E6FA08E6CBF822A5
:0C25B300E0F8A3E0F9A3E0FAA3E0FB22AB
:1025BF007401FF3395E0FEFDFCA3A3A3E02FFFF012
:1025CF00E582158270021583E03EFEF0E5821582EA
:1025DF0070021583E03DFDF0E582158270021583D0
:0525EF00E03CFCF022BD
:0C25F400ECF608EDF608EEF608EFF62213
:0C260000ECF0A3EDF0A3EEF0A3EFF0224D
:10260C00D083D082E493F608740193F60874029395
:09261C00F608740393F6740473CC
:10262500A8828583F0D083D08212263C12263C12E4
:10263500263C12263CE473E493A3C583C5F0C58309
:10264500C8C582C8F0A3C583C5F0C583C8C582C8FF
:012655002262
:0C265600A42582F582E5F03583F583228F
:10266200D083D082F8E4937012740193700DA3A307
:1026720093F8740193F5828883E47374029368601B
:06268200EFA3A3A380DF1B
:10268800EC8EF0A4CCC5F0CCCDF8EFA4CEC5F02DDF
:10269800FDE43CFCE8A42EC8C5F03DFDE43CFCEF9D
:0D26A800A4FFE5F028FEE43DFDE43CFC222B
:00000001FF
